:020000020000FC
:0200000037C007
:100034000C940F2C0C940D2C4156522D436869706E
:100044004261736963322028632920323030362DAF
:1000540032303038204A6F65726720576F6C667291
:04006400616D0000CA
:10007000F894A0E02A2EA1E03A2EA0E1AEBFAFEFA7
:10008000ADBFB0E0A0E0AA95F1F7BA95D9F70E940C
:10009000FB2D0E941B390E943F2FAFEFA09331012F
:1000A0000E940F78A0913C01A370A33009F4AA2705
:1000B000A0933C01442720923D0120923E012092D2
:1000C00050018827789420922D01A0912901A4FD48
:1000D0000C9471000E943F2F0E9495010E944333AF
:1000E000C7CFA1E00E94B52EAA270E946F2E9927A4
:1000F000A7E10E94B02E0E943F2FA0E10E94B02EE7
:10010000C4E0DAE0E7E3F7E10E942B32A7E00E94C7
:10011000B02E0E94E2300704200061D1A6E10E94C7
:10012000B02EC5E0D8E0E6E0F9E00E942B32D8E13D
:10013000F9E10E942B32D8E0F9E0CC5FEC5FC833E4
:10014000A0F366E90E941A336A95E1F70C94A800BF
:10015000A0E00E94B52EA1E00E94C534992720920C
:100160002A01AA270E946F2EA5E10E94B02E0E94AC
:100170003F2FC0E0D0E0EDE1F4E10E947F32A1E545
:100180000E94B02E0E94E230010183838383838327
:10019000204156522D436869704261736963322071
:1001A0008282828282820000A9E9B4E00AE40D938F
:1001B00004EC0D930CE80D9308E20D9302E60D9309
:1001C00006EA0D93509606EA0D9302E60D9308E2B7
:1001D0000D930CE80D9304EC0D930AE40D93E5D117
:1001E00040913D014B3008F0442740933D01642F7E
:1001F00067FD66276B3008F06AE050E06F9302D12C
:100200006F9153955830D1F7A6D17BD150D16F93D0
:100210004FD26F91423E11F46A95EACF433E11F4FA
:100220006395E6CF443E21F4643010F06450E0CF93
:10023000453E21F4673010F46C5FDACF6830F8F097
:100240004A3E11F0443F19F760933D01683039F49C
:100250004A3EE9F6D2D00E94EB1ACFD079CF69306E
:1002600039F44A3EA1F6C9D00E942820C6D070CFEA
:10027000C4D04A3E61F60E949821BFD069CF4F9307
:100280004091140142FD2AC04F914A3E11F0443F73
:1002900041F460933D01B1D088270E949501ADD013
:1002A00057CF413F41F460933D01A7D088270E947A
:1002B0008101A3D04DCF423F39F460933D019DD0E1
:1002C0000E943A1D9AD044CF433F39F460933D01D8
:1002D00094D00E949F1D91D03BCF99CF4F91423F28
:1002E00039F460933D0189D00E946E0386D030CFEF
:1002F000443F99F760933D0180D00E94B6037DD0C2
:1003000027CFA0911601A030E1F70E942A04209285
:100310002D01A0911701A43F09F01ACF06D00E9429
:100320004A33A0E00E946F2EECCF0E943F2F882717
:10033000209216010E94910D209250010E945C2E85
:1003400020922A010E94792FA7E20E94B02E92E00B
:10035000A0913E01A03079F0A33021F4A7E20E94E1
:10036000B02E09C0A0E10E94B02EA0E4A09300012D
:10037000A0EEA0930101A0913E01A03051F40E9493
:10038000E23016002050524553532045534320007D
:1003900021C0A13051F40E94E23069002050524542
:1003A000535320455343200015C0A23051F40E94FE
:1003B000E230420020505245535320455343200021
:1003C00009C00E94E2302F0020505245535320456F
:1003D00053432000A0911601AD3EE1F708950E941D
:1003E000E230FF4156522D43686970426173696380
:1003F000322056302E3832000895A0911601A030D8
:10040000E1F70895A1E0B3E050FDA95F51FDA25FBF
:1004100052FDBA5F4EE2651709F4429540932C01F4
:100420000E94FB300E94E230FF20200040E50E9445
:10043000A62F452F4F5C0E94A62F0E94E230FF207E
:100440002000B3950E94FB300E94E230FF2020D0B4
:10045000D1202000B3950E94FB300E94E230FF20A3
:1004600020D2D3202000E0E0F0E950FDF45F51FD00
:10047000F85E52FDF05DB3950E94FB3066E0459159
:100480000E94A62F6A95D9F7B3950E94FB3066E0CB
:1004900045910E94A62F6A95D9F7B3950E94FB302B
:1004A0000E94E230FF2020202020200008954AE210
:1004B0006A3009F4429540932C010E94E2300F0FFC
:1004C00020202020202000000E94E230100F202059
:1004D000D4D5202000000E94E230110F2020D6D772
:1004E000202000000E94E230120F20494E464F208B
:1004F00000000E94E230130F202020202020000066
:10050000089548E2693009F4429540932C010E9415
:10051000E2300F0820202020202000000E94E2303E
:1005200010082020D8D9202000000E94E2301108B5
:100530002020DADB202000000E94E2301208434F26
:100540004E46494700000E94E23013082020202038
:100550002020000008954CE2683009F44295409351
:100560002C010E94E2300F012020202020200000DA
:100570000E94E23010012020DCDD202000000E94DB
:10058000E23011012020DEDF202000000E94E23056
:10059000120144464C41534800000E94E2301301CE
:1005A00020202020202000000895A0E00E94B02EEE
:1005B0000E94E23015002020202020202020202032
:1005C000202020202020202020202020202020202B
:1005D000202020200000A7E20E94B02E0E94E230DE
:1005E00016002020202020200000A0E60E94B02E2F
:1005F0000E94E23016062045646974200000A0E4E1
:100600000E94B02E0E94E230160C205361766520C5
:100610000000A7E10E94B02E0E94E2301612204C8A
:100620006F6164200000AEE6A0932B07A7E30E9451
:10063000B02E0E94E23016182052756E20000895E8
:10064000A0E00E94B02EA7E20E94B02E0E94E230ED
:1006500016002020202020200000A0E60E94B02EBE
:100660000E94E23016062020202020200000A0E476
:100670000E94B02E0E94E230160C20436F70792049
:100680000000A7E10E94B02E0E94E2301612202046
:10069000202020200000AEE6A0932B07A7E30E94B5
:1006A000B02E0E94E2301618436C65617200089506
:1006B0003DED209217010E94E733409114014470F0
:1006C000431739F0342F403011F46FDFF4CFB8DF27
:1006D000F2CF40911701403071F30895A4E00E94D9
:1006E000B02EC1E0DFE0ECE1F3E10E947F32A0E454
:1006F0000E94B02E0E94E2301002436F70792050A9
:10070000726F6772616D20746F0070913D0160E0DF
:10071000ACE0671709F4A0E60E94B02EB2E1A62F64
:10072000AA0FA60FAD5F0E94FB3040E50E94A62FE6
:10073000462F47704F5C0E94A62F6395683041F7A3
:100740000E944333423E21F47030D1F37A95DFCFDB
:10075000433E21F47730A1F37395D9CF4A3E19F483
:100760000E94417908954D3E59F708950E944937F6
:100770004F436C65617220746869732050726F67B3
:1007800072616D3F2000413009F008950E94227986
:100790000895AA270E94B52EA3E00E94C5348F9326
:1007A00040913D010E9421780E943F2F0E94642EBB
:1007B0009927409116014030E1F70E94E230000095
:1007C0002050524F4752414D200040913D014F5C17
:1007D0000E94A62F4AE30E94A62FC3EDD1E069D262
:1007E00001D30E94E67812D48F91A0E8803069F19D
:1007F000A0ECE6E4F0E1813031F0AFE48A95459178
:100800004030E9F7F8CF5DD292E0A5E0B1E00E9478
:10081000FB300E94DA300E94E230FF20494E205027
:10082000000040913A014F5C0E94A62F4AE30E94CB
:10083000A62FBB27AC2DA3950E94CF2E4AE30E9482
:10084000A62FAD2DA3950E94CF2E0895AAE25A2E71
:1008500070E208959927FADF9CDFD22CAA27BB27E4
:10086000D0922E010E946D330E94E733403E11F476
:10087000AA27F6CF413E11F4AFE12BC0423E11F45E
:10088000AA9527C0433E69F4A3959B2F0E945C095B
:100890009A1730F4BE3511F4AA951BC0AA27B39558
:1008A00018C0443E21F4BA95B7FDBB2712C0463E9E
:1008B00021F4B850B7FDBB270CC0473E11F4B85F18
:1008C00008C0453E11F4B39504C04A3E39F5B395CE
:1008D000AA27A03838F0AFE1BA95B038C0F0AA27FF
:1008E000BB27BECFA03228F0BE3589F0AA27B3952A
:1008F000B7CFBF3508F0BEE50B2F0D1508F4D02E8D
:100900000D2D015F0B1718F40B2F0F50D02E9B2FBE
:100910000E945C099A1708F4A92FA2CF9B2F4E3E84
:1009200039F4AF93BF930E941E09BF91AF919AC152
:100930004F3E39F4AF93BF930E942909BF91AF9105
:1009400091C1493E11F492D18DC14C3E31F4A03099
:1009500009F488CFAA958AD185C1509114015470A9
:1009600009F4D5C0433F51F5A0ECABD10E94E23071
:100970000107524543454956452050524F47524181
:100980004D20592F4E203F007DD1AEF4AFE499D1D8
:100990000E94E2300107524543454956452E2E2E0E
:1009A0002020202020202020202020008DD22ED387
:1009B0004DDF5092C8017DD1882750CF423F39F595
:1009C000A0EC7FD10E94E230010753454E442050F5
:1009D000524F4752414D20592F4E203F000052D1D7
:1009E00056F7AFE46ED10E94E230010753454E4402
:1009F000494E472E2E2E202020202020202000008F
:100A000030922A0193D120922A0120DFD4CF443F93
:100A1000B1F4A0EC56D10E94E2300107434C4541AD
:100A2000522050524F4752414D20592F4E203F00E7
:100A300029D126F4D9D20ADF5092C801BCCF413F58
:100A400041F5A0EC3ED10E94E23001075052494EE0
:100A5000542050524F4752414D20592F4E203F00B5
:100A600011D1B6F4AFE42DD10E94E230010750520B
:100A7000494E54494E472E2E2E2020202020202043
:100A80002000A2E0A0932A0151D120922A01DEDEAB
:100A900092CF433671F462E46093E50165E56093BB
:100AA000E60166E46093E7016DE36093E80177D2C5
:100AB000D9CE483791F462E46093E50165E560932F
:100AC000E60166E46093E7016DE36093E8010E944C
:100AD000CF077AD25092C80118C04637B1F460915E
:100AE000E501623499F460E26093E5016093E60108
:100AF0006093E7016093E8016093E9016093EA0184
:100B000041D284D25092C801ADCE8827ABCE423FAD
:100B100011F5BF93AF93C9D0D9F0A0ECD2D00E9409
:100B2000E2300107534156452050524F4752414D44
:100B300020592F4E203F0000A5D046F40E94B478E3
:100B40000E94E67863D282DE7093C801B2D0882713
:100B5000AF91BF9185CE433FE1F4BF93AF93A5D052
:100B6000B9F0A0ECAED00E94E23001074C4F5354D4
:100B7000204348414E47455320592F4E203F000007
:100B800081D026F70E94E67841D260DE7093C801DA
:100B9000DDCF413F49F46A2E7B2EADD0A62DB72D77
:100BA0005092C8015FCED2CF4D3E09F5BF93AF93AF
:100BB0007CD0A9F0A0EC85D00E94E230010751550D
:100BC000495420572F4F205341564520592F4E202E
:100BD0003F0058D046F7A0911601A030E1F70E94DF
:100BE0005C2EA0E00E946F2EAF91BF910895443F0C
:100BF000E1F45BD029F40E945C2E0E943F2F0895FF
:100C0000AFE65FD00E94E2300107534156452043D2
:100C100048414E474553204245464F524520525584
:100C20004E2100000E94433391CF5091140152FD98
:100C30001CC053FD1AC04C31C0F04038B0F4AF3185
:100C400071F05A2FAFE10E94C2336A916983AA956D
:100C5000A517D9F74883A3955092C80103CE0E94E7
:100C6000C23348835092C801FDCDFCCD0E94C233EF
:100C70005A2F5F3121F0498149935395FACF50E2C1
:100C8000588308950E944333493559F0493749F054
:100C90004A3E39F04E3439F04E3629F04D3E19F0C7
:100CA000F1CF68940895E8940895A091C801A03206
:100CB0000895A0E806D00E94E23001054F4B0000E5
:100CC0000895EF93FF939927A09340010E94E2308B
:100CD000010520202020202020202020202020204E
:100CE0002020202020202020202020202020200024
:100CF000FF91EF910895A0E00E9495334A3E09F4D8
:100D00000895423E21F4A030B9F3AA95F5CF433EB1
:100D100021F4AB3089F3A395EFCF403268F340382C
:100D200058F74883AB3009F0A395E6CFC9ECD1E082
:100D300056E149910E94A62F5A95D9F70E94792F22
:100D40004EE511D016F04A95E1F7542F53954427FC
:100D5000451719F024D04395FBCF43E20E94A62FFC
:100D60000E94792F0895CF93DF935F936F93E89458
:100D7000C4E3D2E053E2459FC00DD11D50E269911A
:100D8000613238F45A95D9F76F915F91DF91CF9125
:100D9000089568946F915F91DF91CF910895DF93EB
:100DA000CF934F935F936F93C1E3D2E053E2459F9C
:100DB000C00DD11DDF93CF93A39653E26A916132A8
:100DC00010F45A95D9F7CF91DF9149910E94A62F3F
:100DD0005A95D9F70E94792F6F915F914F91CF91DA
:100DE000DF910895AF93BF93EF93FF934F93AEE0DE
:100DF000B2E0ECE0FEE04591403011F04D93FBCFC6
:100E00004F91FF91EF91BF91AF910895204578697F
:100E1000742020204E616D6520202053617665206E
:100E20002052656C6F616420202052756E20200076
:100E3000AF93BF93EF93FF934F93AEE0B2E0E8E53B
:100E4000FEE04591403011F04D93FBCF4F91FF9163
:100E5000EF91BF91AF9108952020202020202020E5
:100E60005072696E74202053656E64202020526594
:100E70006376202020204E6577202000AF93BF931B
:100E8000EF93FF934F93AEE0B2E0E4EAFEE04591CA
:100E9000403011F04D93FBCF4F91FF91EF91BF91F7
:100EA000AF9108952041626F72742020202020208D
:100EB0002020202020202020202020202020202032
:100EC0002020202020202000D9DF0E94E2300105D0
:100ED000524543454956494E472E2E2E000020923A
:100EE0002E010E94F4079927E0EEE0934001E3ED24
:100EF000F1E0EE2EFF2E41E10E94CD345CE00E9435
:100F0000E9344B31B9F14A33D1F70E94E9344B311E
:100F100089F1403218F041935A95B9F7403228F0E0
:100F20000E94E9344B3131F1F9CFEEE0F2E0EE2EE0
:100F3000FF2E53E2EE2DFF2DB396EE2EFF2E0E94D4
:100F4000E9344B31B9F04032D0F3433299F006C066
:100F50000E94E9344B3171F0403248F041935A9588
:100F6000B9F70E94E9344B3129F04032D0F793951C
:100F70009036F9F60895A3E2BA9FA1E3B2E0A00D7E
:100F8000B11D0895BF93AF93F6DFC8E7D1E053E2F8
:100F900049914D935A95E1F7AF91BF910895BF9351
:100FA000AF93E9DFC8E7D1E053E24D9149935A95F9
:100FB000E1F7409178014093E90140917901409334
:100FC000EA01AF91BF910895BF93AF934F935F93A1
:100FD000D2DF139640E250E24D935A95E9F75F91C4
:100FE0004F91AF91BF910895DF93CF93BF93AF938C
:100FF0004F9340E2A1E3B2E0CDEFDCE04D932197C7
:10100000E9F74F91AF91BF91CF91DF91DF93CF93EC
:10101000BF93AF934F9341E0A1E3B2E0C0E3D42F7D
:10102000DA5010F0C395FCCFD65CCD93DD93C0E2CF
:10103000CD9390964395403689F74F91AF91BF91EC
:10104000CF91DF910895425245414B004F56455292
:10105000464C4F5700444956494445202F300053D1
:1010600051522046524F4D203C3000434F4E535476
:10107000414E5420544F4F204249470057524F4E43
:10108000472045585052455353494F4E0053594EEF
:10109000544158204552524F5200554E4B4E4F57D7
:1010A0004E204B4559574F52440057524F4E472000
:1010B000464F524D415400424144204C494E454E0A
:1010C000554D424552004E45585420572F4F20460B
:1010D0004F520052455455524E20572F4F20474FE4
:1010E00053554200544F4F204D414E5920474F53C6
:1010F000554200544F4F204D414E5920464F52000B
:10110000493243204552524F5200554E4B4E4F5795
:101110004E204552524F520044464C4153482045C0
:1011200052524F52004F5554204F46204152524187
:101130005900494E434F4D504C4554452050415263
:10114000004B4559574F5244204953204D49535362
:10115000494E470057524F4E472042434F50592067
:10116000004F5554204F462053435245454E0043AF
:10117000414E4E4F54204352454154452046494C20
:1011800045004D454D4F52592046554C4C0046495F
:101190004C45204E4F5420464F554E440050414739
:1011A00045204E4F5420494E2046494C4500504161
:1011B000474553204E4F5420494E2052414E4745FB
:1011C000004E4F5420494E20475241504849435306
:1011D000204D4F4445004E4F5420494E2054455811
:1011E00054204D4F4445004E4F2055535220464900
:1011F0004C4500535243204F5554204F46205343F3
:101200005245454E0044455354204F5554204F46B7
:101210002053435245454E0057524F4E472053509E
:101220005249544500494F2044495341424C45449A
:10123000004E4F204558544D454D0000BE3508F036
:101240000895BF9328D0B395BE35E1F7BDDEBF91B9
:10125000DDCEBE3508F00895BF93AF93AB2FAA95AE
:10126000BDE508D0BA95BA17E1F7B395ADDEAF91F9
:10127000BF91CCCEBF93AF93DF93CF937CDE139619
:10128000ED01B0E2A991AAA3BA95E1F7CF91DF9160
:10129000AF91BF910895BF93AF93DF93CF936BDE70
:1012A0001396ED01B0E2ABA1A993BA95E1F7CF9106
:1012B000DF91AF91BF910895BF93AF93DF93CF9329
:1012C0005ADEED0193964E914132E8F34038D8F75B
:1012D000AC1BBC0B9A2F925097FD9927CF91DF91B1
:1012E000AF91BF910895CAEEDCE02A922A9280E085
:1012F0002F92AA27BB27442771917032E9F37C31E2
:1013000021F4A191BB27719156C07E3121F4A191A6
:10131000BB27719150C07D3121F4B191A1917191A0
:101320004AC07F3121F4B191A191719144C07C31C7
:1013300030F4572F4C2E5D2ECE2FDF2F63C074322A
:10134000C1F47191703320F07A3310F4705305C0FA
:10135000713468F0773458F47753B03148F4A2957B
:10136000B2955A2F5F70A07FB52BA70FEACF23C08D
:1013700029C0703350F17A3340F5403810F086E0E0
:1013800027C1AA0FBB1FF0F04A2E5B2EAA0FBB1F6E
:10139000C8F0AA0FBB1FB0F0A40DB51D98F0705394
:1013A000A70FB21D78F0B7FD0DC07191703318F022
:1013B0007A3308F4E6CF4F3709F470D1AA93BA9381
:1013C00040E89DCF85E004C144C07134E8F37B352B
:1013D000D8F76081613458F16B3548F54C2E5D2E9D
:1013E000CE2FDF2F21970C2F1D2FE6ECFAE152E0D4
:1013F0007591703011F488E0EBC0703261F469913E
:10140000683299F45F93452FAA27BB27EC2FFD2F55
:10141000C42DD52D71CF6991671751F37591703235
:10142000E9F75395C02FD12FE3CF87E0D1C04038E3
:1014300010F086E0CDC07154770FEF93FF93E0E991
:10144000FCE0E70FF21DA191B191FF91EF91719135
:10145000B2CF7D3251F44F3711F444274DCF20F4F1
:10146000403210F04FE748CF6CC0783231F471E071
:101470007F93AA27BB27472F3FCF793209F05BC064
:101480005F91513019F0523011F400D150C05330F7
:1014900011F410D14CC0543029F4C9D1803009F076
:1014A00097C043C0553029F4B991A991B095A09542
:1014B0003CC0563009F4DAC1573009F46DC25830D7
:1014C00009F47EC2593009F493C25A3009F4A9C212
:1014D0005B3009F4B1C25C3009F4B2C25D3009F48A
:1014E000B4C25E3009F48EC2503109F4EAC1513100
:1014F00009F422C1523109F425C1533109F4EEC176
:10150000543109F403C25F3009F4CBC2553109F4F8
:10151000B9C1563109F4CDC1503029F06ED08030B8
:1015200009F056C0ADCF86E00895AA93BA93AA27D2
:10153000BB2742E0E1CE4F3720F44F3010F086E079
:1015400047C07C3361F471E260816E3319F472E25A
:10155000619142C06D3311F473E261913DC07E33FD
:1015600039F474E260816D3311F475E2619134C035
:101570007D3311F476E230C07B3211F470E32CC07D
:101580007D3211F471E328C0733211F472E324C088
:101590007A3211F470E420C07F3211F471E41CC07F
:1015A000753211F472E418C0763211F473E414C089
:1015B0005F91503021F05F3130F01FD0F9CFB991F9
:1015C000A9913197089586E05F915030C1F3FCCF27
:1015D0004F914030E9F708955F91A72FB52FA07F75
:1015E000B07FBA1720F009D0803091F7F5CF5F9324
:1015F0007F93AA27BB27472F7FCE5F934F931991E5
:101600000991B991A991513211F4FED03AC05232E8
:1016100021F4F3D0A150A17034C0533221F4FCD096
:10162000A150A1702EC0543211F4F6D02AC0553208
:1016300021F4EAD0A150A17024C0563211F4DDD0BB
:1016400020C0503311F441D01CC0513311F43CD0B0
:1016500018C0523319F4A02BB12B13C0503411F41D
:101660003FD00FC0513411F4A7D00BC0523421F435
:10167000A3D0A22FB32F05C0533419F4A023B12354
:1016800000C0AA93BA934F915F910895B991A9911F
:1016900003D0AA93BA930895B7FF0895A095B09583
:1016A000A30DB21D089517FF089500951095030D21
:1016B000121D0895B991A991AB2B29F0B7FBA1E0B8
:1016C000BB270EF41297E5CFF0DF2B2F2127A00FB9
:1016D000B11F27FD08952B2F212727FD82E00895B4
:1016E0000CD0A22FB32FBF770EF4D8DF37FD03C085
:1016F000452B09F4089582E008957AD0CDDFB19F9B
:10170000402D512DA09F202D312DA19F300D411D29
:10171000521DB09F300D411D521D089508E611E085
:10172000B03818F0A00FB11FFBCFA017B10718F009
:10173000A01BB10BFACF0895B991A9910AE5A01B9E
:10174000B20902C0B991A991E9DFFF93EF93E4E6F2
:10175000FAE70AE510E0A017B10748F4E00FF11F1F
:10176000EA1BFB0BA491EF91FF91BB27DECE04EBAC
:1017700010E0A017B10778F40AE510E0E01BF10BC8
:10178000EA0FFB1FA491EF91FF91BB27A095B095A5
:10179000A30DB21DCACE0EE011E0A017B10728F4C8
:1017A000E00FF11FEA1BFB0BEDCF0EE011E0E01B99
:1017B000F10BEA0FFB1FD6CF212F202B11F483E072
:1017C000089516D022273327442751E1441FAA1F2A
:1017D000BB1F5A9551F0221F331F4FEF201B310BB7
:1017E000A8F7200F311F40E0F1CF0EF457CF089536
:1017F0002B2F212727FB50DF56CF0A271B27AA278D
:10180000BB27012B89F00895B0581058A01BB10BCD
:10181000AA27BB2748F00895B05810580A1B1B0B85
:10182000AA27BB2708F00895A1E0B0E00895B99178
:10183000A99184E0B7FD08950F931F932F933F93D1
:1018400088270A2F1B2FB2E0AA27232D3327021B3C
:10185000130B20F0A3952B0F321DF9CFBB27AA93B2
:10186000BA933F912F911F910F9108954F935F93DA
:101870000E9400351991099142DFA42FB52F5F9185
:101880004F9153CE19910991023039F420925001B1
:10189000A2E0A0933301BB2748CE013031F4A091E0
:1018A0003301A03011F430923301A0913301BB27F2
:1018B0003CCE199109910EBD0E944C17AEB5BB27C5
:1018C00034CEB991B0937301A991A0937201CF93D3
:1018D000DF930E945017DF91CF9127CEB991A99144
:1018E000BF3F71F0A09358010E940820803021F082
:1018F000AFEFBFEF882719CEA42FBB270C94950A12
:101900000E940D208827B42FAA270FCEB991A99144
:10191000BF3F21F5A0FD11C0DF93CF93FF93EF935D
:101920000E940520803019F08827CC27DD27DE01B2
:10193000EF91FF91CF91DF91F8CDDF93CF93FF939C
:10194000EF930E940520803019F08827EE27FF27AB
:10195000DF01EF91FF91CF91DF91E7CDA093580187
:101960000E940820803021F08827AA27BB27DDCDE0
:10197000DF93CF937F9377270E941020DF3F41F4BE
:10198000CF3F31F4A72FBB277F91CF91DF91CDCDF2
:101990007395703889F7F6CFA991A991A770A06CBB
:1019A000A0937C00A0917A00A064A0937A00A091FB
:1019B0007A00A6FDFCCFA0917800B0917900B5CD5A
:1019C000B991A991B03061F4AF3F79F0A770A395B8
:1019D000B0B1B695AA95E9F7AA27AA1FBB27A5CD4E
:1019E000BA2FA0B1AB23BB27A0CDA0B1BB279DCD03
:1019F000B991A99171E00E9462398030C9F4BB2786
:101A0000A52F93CDB991A991CF93DF93CA2FDB2F47
:101A10000E949F39DF91CF91803051F4BB27A42FD2
:101A200084CDA99179910E947D39803009F47DCDD2
:101A3000AA27BB278FE0C8CDB991A991BB2775CD47
:101A4000B991A991AB2FBB2770CD0F93B991099193
:101A5000AA27BB27037039F40091140100FD1196E9
:101A600002FD11971CC0013039F40091140101FDF1
:101A7000119603FD119713C0023049F4009116012D
:101A8000023E09F41197033E51F4119608C00091EB
:101A90001601043E09F41196053E09F411970F91C1
:101AA00044CDB991A991BB27A13021F4A0916D013A
:101AB000A3953BCDA23021F4A0916E01A39535CD25
:101AC000A0916F0132CD4142532053474E205351D4
:101AD00052204E4F5420524E442041444320494E00
:101AE00020585045454B2054454D50204C4F2048E0
:101AF00049204B455920455045454B2045525220E1
:101B000041522053494E20434F532046545950458B
:101B1000204653495A45205053544154205350496C
:101B20002000FCE0E0E9A0E0B4EBA193BA95E9F76E
:101B3000F1E0E8E6B0E1A193BA95E9F7FDE0ECE366
:101B4000B0E0A193A193A193BA95D9F7DD24CC2459
:101B500020920F01AEE0A0932C01ACE3A0934401CE
:101B6000AEE2A0934501AFEFA09377010E943F2F13
:101B700020925001A2E0A0933301A6ECA0937A003A
:101B800040913D0140933A01409337010E942178F2
:101B90009C2D0E943D781FD0803039F4AC2DAF359C
:101BA000B8F39CE0209250010895C0926D01D0924C
:101BB0006E0180936F0120925001409177014F3563
:101BC00020F4DD24C42E8827E3CF9CE0209250012E
:101BD0000895F70129C0F1E0E0EA20922A01882760
:101BE000AD2DBB27AB1701F171917F3FB1F17C3176
:101BF000C9F07E31B9F07D31A1F07F3191F07732BB
:101C000061F1723241F471917F3F39F1773229F1FC
:101C10007232C9F7E9CF7A3339F7B395AB1721F7A9
:101C200003C071917191E0CF70912D0170FF05C0DB
:101C300081E07E7F70932D01089572FF09C0AB7F14
:101C400070932D01A0913E01A03011F40E94A51ABD
:101C50000E94E73371917F3F19F4DD24C394089506
:101C600077FD2BC0703201F37A3311F4D394DCCFBB
:101C7000773299F37134D8F07B3528F07052713493
:101C8000B0F07B35A0F4672E0E948B167D3379F47B
:101C90002ADB803069F4762D7154770FDCE0C0E9DF
:101CA000C70FD21DA993B99395CFEF91FF9187E00C
:101CB0000895703810F487E08CCF7F01E4E6FEE0F1
:101CC0007F73E70FF21D099445C0EDC096C236C17F
:101CD0000CC1DFC220C300C728C329C32DC330C332
:101CE00040C349C34EC3A4C3CAC2FCC32CC46EC103
:101CF0006EC47EC483C4DFC18BC288C493C49AC43B
:101D00005BC540C1D5C06DC21FC0E3C49DC418C32C
:101D1000E4C405C544C2CFC2C6C56CC718C624C634
:101D200029C669C16CC6BBC63DC72AC639C650C2E2
:101D300016C559C615C177C299C3F2C294C49AC4D4
:101D400033C16BC13DC688C188E0089584E1089520
:101D500083E108950E948F169CE0732C20922A0143
:101D6000B191B032E9F3BA3311F0BF3F59F4319772
:101D700070FC0E94792F40912A01443010F00E949B
:101D8000223928CFBB3311F47724EACFBC3291F447
:101D900040912A01403031F40E94A52FBA2DB7702E
:101DA000D9F706C00E94A52FB0912B01B770D1F7CB
:101DB0007724D6CF732CB332C9F4209258012092E5
:101DC000590191DA4A2F40932A01443018F44330E4
:101DD00001F4C6CF0E942639683051F550912A018E
:101DE0005E7F0E942839683119F5BACFB03411F5F9
:101DF00062D740912A01433018F40E94FB30B0CFE3
:101E000039F4A0935801B0935901A0932B01A8CFA6
:101E10005FEF0E942839683259F45A2F0E942839FE
:101E2000683231F45B2F0E942839683209F498CF68
:101E30008FE00895B13229F456DA9A2F91CF97CFD7
:101E40008FCFB23241F441914F3FC9F34232C1F3D7
:101E50000E94A62FF8CFB63291F445DAB33010F0D5
:101E600082E10895CCE3DDE0CA0FDB1F49914030E9
:101E700029F00E94A62F1196B330C0F371CFB5326E
:101E800029F431DA4A2F0E94A62F6ACF31972BDA34
:101E9000803009F00895903818F40E94CF2E60CF5A
:101EA0000E942A2F5DCFA0E0B8D60E943F2F91CE8E
:101EB000A2E0B3D6A030C1F0A13059F0A0915A01F0
:101EC000A770AA0FB0912C01B770A295BA2BB0934E
:101ED0002C01A0915801A770AA0FB0912C01B07FDE
:101EE000BA2BB0932C0175CE33CFA3E096D6A33096
:101EF00018F1A0915801B0915901A0937201B093CB
:101F00007301A0915A01B0915B01A0935801B09365
:101F10005901A0915C01B0915D01B03011F4A03085
:101F200051F00D010E9450170E94E416D00180303C
:101F300021F41197F2CF4DCE0BCF0895A5E06DD6C9
:101F4000A43068F078D77F93A5D6E0936B01F09327
:101F50006C010E9409327F9170932C013ACEF8CE29
:101F6000A5E05BD6A43068F066D77F9393D6E09364
:101F70006B01F0936C010E942B327F9170932C01C6
:101F800028CEE6CEA5E049D6A43068F054D77F939A
:101F900081D6C0936B01D0936C010E9496367F91DD
:101FA00070932C0116CED4CEA5E037D6A43068F0BD
:101FB00042D77F936FD6C0936B01D0936C010E9480
:101FC000E6367F9170932C0104CEC2CEA3E025D6D5
:101FD000A23080F030D77F93B0915801A0915A0180
:101FE000A0936B01B0936C010E940E317F917093AE
:101FF0002C01EFCDADCEA5E010D6A43068F01BD7F4
:102000007F9348D6E0936B01F0936C010E94E53218
:102010007F9170932C01DDCD9BCEA0913E01A0302D
:1020200011F08CE10895A1E0F8D5A130A8F3A091BA
:102030005801B0915901CCE3DDE0CA0FDB1F40919C
:102040002C014F93AF92BF920E942D37BF90AF905B
:102050004F9140932C01BDCDA0913E01A03011F0D5
:102060008CE1089541D6C0937001D093710153D68D
:102070007C32F9F4A1E0D2D5A13070F2A0915801E0
:10208000B0915901CCE3DDE0CA0FDB1F40912C0178
:102090004F93AF92BF920E945637BF90AF90C091BE
:1020A0007001D0917101499329924F9140932C0175
:1020B00090CD87E08ECDA0913E01A03011F08CE153
:1020C000089512D6C0937001D093710124D67C324A
:1020D00081F7A1E0A3D5A13009F03ACEFF93EF93A9
:1020E000AF92BF9240912C014F937F934F704093DA
:1020F0002C010E941519C1E0D2E0ECE1F5E10E944B
:102100007F32C0912C01C295C0932C010E94E23015
:1021100003020000A0915801B0915901CCE3DDE029
:10212000CA0FDB1FA6E14991403230F0403820F45D
:102130000E94A62FAA95B9F7772761E025D00E94C3
:102140003419623079F4C0917001D09171017993A2
:1021500029927F914F9140932C01BF90AF90EF91C6
:10216000FF9137CD7F914F9140932C01BF90AF905D
:10217000EF91FF91C0917001D09171014FEF4993A0
:10218000499327CD87E025CD0E942F1788276030FF
:1021900009F408950E94DE1D882762E00895A3E0F7
:1021A0003CD5A230A0F047D67F93D0916C01C0916E
:1021B0006B01F0915801E0915A01E0936B01F093AB
:1021C0006C010E94E5327F9170932C0102CDC0CD4D
:1021D000A4E023D5A43021F45DD50E94E131F9CCEF
:1021E000B7CDA1E01AD5A13090F0A0915801A295E9
:1021F000AA0FAF7EA0930F01ECCCA1E00ED5A130C9
:1022000030F0A0915801A150CA2EDD240895A0CD30
:10221000A1E003D5A130D8F3A0915801A150A0931B
:102220007701D7CC95CDA5E0F8D4A23030F1F1E01C
:10223000E0915801E770B0915A01B770BB0FB295A9
:10224000B193A230C9F0E770B0915C01B770BB0FD9
:10225000B295B193A33081F0E770B0915E01B77091
:10226000BB0FB295B193A43039F0E770B091600123
:10227000B770BB0FB295B193ACCC6ACD69CDA1E07C
:10228000CCD4A130D8F3A0915801A3700E946F2E36
:10229000A0CCA1E0C2D4A13068F0A0915801B091C7
:1022A0005901B03019F4A03009F493CC0E941A33CC
:1022B0001197F7CF4DCD20925001A2E0A0933301AA
:1022C000A3E0ABD4A33020F1CCE3DDE0A091580132
:1022D000B0915901B330E8F4AC0FBD1FA093520187
:1022E000A0935401B0935301B0935501A0915A01AA
:1022F000B0915B01B33068F4AC0FBD1FA0935601E1
:10230000B0935701A0915C01A0935001209233013A
:1023100060CC82E15ECC20925001BF91BF910895C4
:1023200000D5AB2B09F499CC55CCF9D453CCF7019B
:10233000C2D40E94FB304ECCF4D40E9423334ACC4A
:10234000672F6F93EED46F914A2F0E94A62F65FDE1
:102350000E94CB33E1D47C3271F7DDD40E94730943
:10236000F3CFC2D420921701A0911701A030E1F35E
:10237000A99329922FCCB8D4A0911601A9932992A0
:1023800029CCA2E04AD4A13019F0A23021F1E0CC4E
:10239000A0915801AA95AF3510F08AE01ACCB091FF
:1023A0006901BF3010F08DE014CCAF93CCEEDCE0CF
:1023B000A5E0AB9FC00DD11DB395B0936901BD2DB4
:1023C000B395B068B993BC2DB993B0913D01B99361
:1023D000DD24CF900895A0915A01AA95AF35E8F673
:1023E000B0915801BA95B770B0933701B0916901B7
:1023F000BF3010F08DE0EDCBAF93CCEEDCE0A5E08C
:10240000AB9FC00DD11DB395B0936901BD2DB395A0
:10241000B068B993BC2DB993B0913A01B993DD245A
:10242000CF904091370140933A010E94217808955E
:1024300076D4B0916901B03011F48CE00895BA956A
:10244000CCEEDCE0A5E0AB9FC00DD11DB0936901DF
:10245000B991B7FFF2CFBF77DB2EC9904991409376
:102460003A010E942178089587E0089558D453D402
:102470007134D0F37B35C0F77154770F672E4BD48E
:102480007D3391F70E947309803009F00895DCE0F4
:10249000C0E9C60DD21DA993B9933DD4743521F777
:1024A00071917F3409F70E9473094A2E5B2E8030A8
:1024B00009F00895B0916901BF3010F08EE00895E1
:1024C000CCEEDCE0A5E0AB9FC00DD11DB395B09381
:1024D0006901BD2DB395B993BC2DB9936992499209
:1024E000599278CB1CD4B0916901B03011F48BE0D3
:1024F0000895BA95CCEEDCE0A5E0AB9FC00DD11DF0
:10250000B991B7FDF4CFBF77B0936A015990799133
:10251000BCE0A0E9A70FB21D0D911D91030D121D86
:102520001E930E93A991B99111960A1741F41B17A6
:1025300031F4B0916901BA95B09369014BCBC52CC8
:10254000D0906A010895A0913E01A03011F08CE175
:102550000895E5D3BFEFB0937801B191B032E9F3BC
:102560004B2FBF3F21F40E94792F319733CBBA33E1
:10257000D1F3BB3391F3BC3231F40E94A52FBA2DB5
:10258000B770D9F7EACFB23241F441914F3F59F3D6
:10259000423219F30E94A62FF8CFB134B0F0BB3508
:1025A000A0F4B154BB0FB0936A01B081B13418F0FC
:1025B000BB3508F40AC0B8D3DCE0C0E910916A0169
:1025C000C10FD21DA993B993C8CF87E00895A9D3AD
:1025D000803009F0FFCA4A2F4B2BE1F340912201D2
:1025E0004030E1F3409122014030E1F71197F3CF01
:1025F00098D3A0932301B0932401EDCF75D3A0917C
:102600002301A993A0912401A993E4CA8AD34A2F54
:102610000E94CD3481D37C3221F47DD30E94730992
:10262000F6CFD8CA0E94D934A42FBB275DD3A99373
:10263000B993D0CAF7014BD34A2FD73020F4C03D0D
:1026400010F40E94A839C6CAF70141D35A2FAC2F03
:10265000BD2F71E00E9470390E941A330E941A3314
:102660000E941A33B7CA70910D0170FD30C059D362
:10267000A1B9B0CA70910D0170FD29C0F70127D32F
:10268000D030B1F4BC2FB770B39577276FE7A0FDBA
:1026900070E8A0FD6FEF77FB770F70F967FB660FAF
:1026A00060F9BA95C1F702B1072B062302B992CAA5
:1026B000D13041F4B2B1C095BC23C095CA23BC2B24
:1026C000B2B988CAD230E9F70E943D1783CA82E2C4
:1026D000089527D30E94C5347DCA06D3C0937001E4
:1026E000D093710109911991105815D37C32A9F436
:1026F000EED2B058D058C017D10710F00C2F1D2FB4
:10270000A017B10710F40A2F1B2FD0917101C091AF
:1027100070011058099319935DCA86E00895A0913D
:102720003E01A03011F08CE10895DED2C09370011B
:10273000D0937101F0D27C3281F7BDD2C8ECD1E0E8
:102740007EE17B9FC00DD11DCA0FD21DBB27A88182
:10275000D0917101C0917001A993B9933BCAA09126
:102760003E01A03011F08CE10895BED2C0937001FB
:10277000D0937101D0D27C3281F69DD2C8ECD1E0E9
:102780007EE17B9FC00DD11DCA0FD21DA2EBCA0FE7
:10279000A2E0DA0FBB27A881A695BA2FA777B2953A
:1027A000B078AB2BBB27D0917101C0917001A99378
:1027B000B99310CA86E0089597D2C0937001D09360
:1027C0007101A9D27C32B1F776D2C8ECD1E0709118
:1027D0003E017370703021F5AF93BF93A695B69507
:1027E0007EE17B9FC00DD11DCA0FD21D7881BF91A4
:1027F000AF91A0FD7695B0FD7695B0FD7695A2EBF4
:10280000B2E0CA0FDB1FAC9170FDA295A695A77030
:10281000BB27D0917101C0917001A993B993DAC916
:102820007130D1F4AF93A695A695A69575E17B9FDF
:10283000C00DD11DCA0FD21D7881AF91A2FD729536
:10284000A1FD7695A1FD7695A0FD76957170D1E0FC
:10285000C72FA881A295DACF7130F1F7AF93A69573
:10286000A6957EE17B9FC00DD11DCA0FD21D788138
:10287000AF91A1FD7295A0FD7695A0FD7695737040
:10288000D1E0C72FA881A295C1CFAF93A6957AE2D8
:102890007B9FC00DD11DCA0FD21D7881AF91A0FDC5
:1028A0007295A72FB3CFA0913E01A03011F08CE11B
:1028B0000895A3E0B2D1A33080F0A0915801B09167
:1028C0005901B33010F082E10895B23039F4A73FD6
:1028D00028F082E1089581E208953ACACCE3DDE070
:1028E000CA0FDB1FC0934601D0934901AC81A030D1
:1028F00091F3AE3180F7BB81B03069F3B73158F74F
:10290000C0915801D09159012596BA9F000C111C15
:10291000000C111CC00DC11DD330E8F6D0915A0136
:10292000C0915C01C0934801D0934B01CF3F51F05F
:10293000DF3F41F0CA0FCA95CE3138F4DB0FDA958C
:10294000D73118F40E94C83744C986E10895A09190
:102950003E01A03011F08CE10895E1D1A0912D014C
:10296000A460A0932D0136C9A0912901A062A09373
:10297000290130C9A0912901AF7DA09329012AC95D
:10298000A3E04BD1A33009F0E3C90E9408204431F1
:1029900011F08EE108950E941C208030D9F719C9EA
:1029A000A3E03BD1A33009F0D3C90E9408204431F1
:1029B00011F08EE108950E941F208030D9F709C9D7
:1029C000A2E02BD1A23009F0C3C9A4E1A0935C011D
:1029D0000E941620803009F4FCC808950E94192036
:1029E000803059F4F6C8A1E018D1A13009F0B0C97F
:1029F0000E940820443191F38EE108954EC0F70102
:102A00003ED1A09374010E9426396830B9F790FF37
:102A100028C0592F0E942839603481F7A030C9F0AE
:102A2000DDE0CCE3409174014B0F4A1BC40FD21D73
:102A3000A13039F00E942C39603579F55883AA9578
:102A4000EFCF0E943139683541F558830E94223911
:102A5000C1C80E942C395030A1F350937401A52FA6
:102A6000DFCF592F0E9428396831B9F43A2FDDE0C1
:102A7000CCE3409174014B0F4A1BC40FD21D588107
:102A8000503011F4303031F00E942839683229F486
:102A9000AA9569F70E9422399DC88FE0089541D117
:102AA000A0935801B093590137D17C3249F4319643
:102AB00032D1723231F031970E94730985D1F4CF4F
:102AC00089C87191723231F07F3F21F0BB27A72F67
:102AD0007BD1F7CF7081E8CFA0913E01A03011F4F7
:102AE0008DE10895A7E099D0B0915801B0934C01C1
:102AF000B13039F0B23009F1B33009F43CC085E1AE
:102B00000895A730E1F7C8E5D1E0BA81B093490153
:102B1000BC81B0934601BE81B0934A01B885B093A1
:102B20004701BA85B0934B01BC85B09348010E9420
:102B30002535803009F008954CC8A63001F7C8E566
:102B4000D1E0BA81B0934901BC81B0934601BE8106
:102B5000B0934A01B885B0934701BA85B093480154
:102B6000BB85B0934B010E942535803009F0089554
:102B70000C94E90DC4CFA430E9F7C8E5D1E0BA81DF
:102B8000B0934601BB81B0934901BC81B0934B0126
:102B9000BE81B09348010E942535803009F0089528
:102BA0000C94E90DA0913E01A03011F08CE1089544
:102BB000F7018DD0C0935801D09359015091740101
:102BC000A51708F45A2FA8E7B1E0503071F04D91E5
:102BD000A0937501B0937601A42FBB27F5D0A091E7
:102BE0007501B09176015A95F0CFAA27BB27ECD09A
:102BF0000C94EA0DA0913E01A03011F08CE10895F3
:102C0000A1E00BD0A13040F0A09158014A2F4370B1
:102C10000E9496380C94E90D9BC8F701A03009F486
:102C20000895DF93CF93C8E5D1E040E05A2F5030AC
:102C300029F4A42F7F01CF91DF910895DF93CF93E3
:102C40004F935F930E9473095F914F91CF91DF91F2
:102C5000893121F488277F01A42F0895A993B9937E
:102C600043955A95503019F371917032E9F37C32E3
:102C700029F33197A42F7F01CF91DF910895A3E02D
:102C8000CCDFA33009F590915801B0915A01A09181
:102C90005C010895D0915801C0915A01F0915C01F6
:102CA000E0915E01C0934601D0934901E093470152
:102CB000F0934A010895A2E0B1DFA23029F4B09167
:102CC0005801A0915A010895AF91AF9141C8A2E077
:102CD000A5DFA230C9F7C0915801D0915901A09148
:102CE0005A01B0915B010895F70115D0713478F065
:102CF0007B3538F47154770FDCE0C0E9C70FD21D83
:102D00000895713620F07B3710F47156F4CF8F910F
:102D10008F9187E0089571917032E9F30895F7017A
:102D20000895F7010C947309EF93FF930E94AF335A
:102D3000EC2FFD2F00E00E944F3370912D01713078
:102D400011F4872F08C04A3EC9F400937401003083
:102D500031F4AA27BB278827FF91EF910895C8E790
:102D6000D1E0A191A9930A95E1F7A0E2A993AFEF71
:102D7000A993E8E7F1E00E947309EDCF4C3E49F4D6
:102D80000030C9F2AA940E94AF33A0E2A8830A954A
:102D9000D2CF403248F24B3738F6AA2DAD3120F66B
:102DA0000E94A62F0395C7CF92E0BB27AC2DA39519
:102DB0000E94CF2E4AE30E94A62FBB27AD2D0E9472
:102DC000CF2E0E94A52F0895DF93CF93BF93AF938B
:102DD000A0915801B0915901B33098F4CCE3DDE0F3
:102DE000CA0FDB1FAF91BF91A883C0915801D0914A
:102DF00059012196C0935801D0935901CF91DF9189
:102E00000895B45090F0AA0FBB1FB33070F4CCE318
:102E1000DDE0CA0FDB1FAF91BF91A993B993C091B9
:102E20005801D09159012296E5CF82E1AF91BF912F
:102E3000CF91DF91089570912C01A0FF0895A330E8
:102E400059F450915C015F70550F707F572B709152
:102E50002C0150932C01089550916001F4CF0E94F1
:102E60002220403011F466270895409360010E94AB
:102E70001320413009F066270895AF3F31F42C9AB2
:102E80002CBCACE5ACBD3DBC08952CBCAF73A064BC
:102E9000ACBD3DBC2C980895BDB5B7FFFDCF0895DE
:102EA0005091720140917301433038F4DDE0CCE37E
:102EB000C50FD41FA991BB2710C05050444058F0F3
:102EC000550F441F433038F4DDE0CCE3C50FD41F69
:102ED000A991B99102C082E1089540917201509187
:102EE0007301430D521D4093720150937301803062
:102EF00009F408954F914F910895A0EAB1E04FEF82
:102F000052E24D935A95E9F7C8E9D1E040E25A916F
:102F1000503211F44A95D9F7442EA0EAB1E0C8E73F
:102F2000D1E04C0EA03C28F4C41518F44881403080
:102F300009F4089593D04F3FE1F37AD04F3FC9F39E
:102F4000403081F798D0403069F73DD0403051F79C
:102F50000AD0403039F74991413618F04B3708F420
:102F600040524D93DFCF4881403320F04A3310F474
:102F7000405302C044270895642F77272196488143
:102F8000403380F04A3370F44053660F771F0B01D3
:102F9000660F771F660F771F600D711D640F721D1E
:102FA0002196EDCF703029F04DE14D937D936D93D7
:102FB00008956A3020F04CE14D936D930895605D63
:102FC0006D934CE108954881443211F044270895EF
:102FD00066277727219658815033F8F05A3310F43A
:102FE00050530BC05134C8F0573410F4575305C038
:102FF000513698F0573688F457555F705295550FF3
:10300000661F771F550F661F771F550F661F771FA7
:10301000550F661F771F2196DECF703029F04FE1E4
:103020004D937D936D9308954EE14D936D93089567
:103030004881423211F04427089521964D934991D9
:10304000423219F44D9341E00895403029F442E2B0
:103050004D934FEF4D9308954D93F1CF48814732F3
:1030600011F04427089521964D9349914030E1F79E
:103070004FEF4D930895FF93EF93BF93AF935F93FB
:10308000E8E5F4E40E014591403089F0689457E09A
:10309000A591AE3239F0B991B13608F0B052AB1704
:1030A00009F0E8945A95A1F716F0E001EBCF5F9193
:1030B000AF91BF91EF91FF91403041F04D934F930D
:1030C0004881403211F42196FBCF4F910895CBE710
:1030D000D1E0A0EAB1E040E2E0E24993EA95E9F705
:1030E000A097A03C29F04D91423010F04F3F11F4D1
:1030F00029920895403220F0403810F486D0F1CF64
:103100004C3121F4ED91FF2719D0EBCF4D3121F453
:10311000FD91ED9113D0E5CF4E3131F444E275D0FD
:10312000ED91FF273CD0DDCF4F3131F444E26DD03B
:10313000FD91ED9134D0D5CF50D0D3CFE8944FE26C
:103140004395E051F742E0F7E05FF84D403311F06E
:1031500063D068944FE24395E85EF340E0F7E851AE
:10316000FC4F16F0403311F057D068944FE243956E
:10317000E456F040E0F7EC59FF4F16F0403311F001
:103180004BD068944FE24395EA50E8F7E65F16F0BB
:10319000403309F041D040E34E0F3ED00895E8940B
:1031A0004F2F42954F7011F012D068944F2F4F70EF
:1031B0000EF011F00CD068944E2F42954F700EF027
:1031C00011F005D068944E2F4F7001D00895405DE6
:1031D0004A3308F0495F20D00895E8E5F4E45591BA
:1031E000503009F40895451711F03796F8CF5F93E2
:1031F00057E045914E3209F00FD05A95D1F75F91C3
:103200005C3110F040E208D008954993CB3918F0B2
:1032100029924F914F9108954993CB3928F02992E3
:103220004F914F914F914F910895FF93EF93A0913C
:103230002C01A0935101A0910F01A0935401A091E2
:103240002A01A093500120922A01E8ECF1E0CCE29F
:10325000D7E0BEE2AEE141914993AA95E1F7BA9574
:10326000C9F7EF91FF910895FF93EF93A091540157
:10327000A0930F01A0915101A0932C01A0915001A6
:10328000A0932A01ECE2F7E0C8ECD1E0E2CFA091F4
:103290000D01A0FD35C0C6E0D4E0A9E4BFE441B112
:1032A00058E040FDB99340FFA99346955A95C9F758
:1032B000C4E2D4E0A0E3B1E340B158E040FDB993EB
:1032C00040FFA99346955A95C9F7C8EBD6E0AFEAF7
:1032D000BFE241B158E040FDB99340FFA993469544
:1032E0005A95C9F7C6EDD6E0A0E8BEE440B158E073
:1032F00040FDB99340FFA99346955A95C9F70895A3
:103300000E94E230130020494F2044495341424C6F
:10331000454420000895452FA6E10E94B02E4F5B42
:103320000E94A62F4DE30E94A62FA7E10E94B02E77
:10333000C0E9DCE0C50FD21DC50FD21DA991B9911E
:103340009DE00E94CF2E0895A3E10E94FB30A5E0EE
:10335000C62FCA95AC9FCCEEDCE0C00DD11DA88174
:10336000A7FF0AC00E94E230FF43414C4C202000DE
:10337000A981AF770EC008950E94E230FF464F52F8
:1033800020004A8146954F5B0E94A62F0E94A52FE0
:10339000A981BB27A39592E00E94CF2E4AE30E9409
:1033A000A62FBB27A8810E94CF2E089520920F013F
:1033B000A7E00E94B02E0E943F2F0E94E230120030
:1033C00042495420303132333435363700000E94C0
:1033D000E2301300444952000E94E23014004C4590
:1033E0005600A7E20E94B02E0E94E230160020454F
:1033F000786974200000A0E60E94B02E0E94E2309E
:1034000016062020476F20200000A0E40E94B02E66
:103410000E94E230160C2053746570200000A7E172
:103420000E94B02E0E94E230161220566965772065
:103430000000AEE6A0932B07A7E30E94B02E0E94E7
:10344000E2301618202020202000A5E00E94B02E97
:103450000E94E23000004156522D4368697042617B
:1034600073696332204D4F4E202020205000409140
:1034700037014F5C0E94A62F0E94E230FF3A000005
:1034800092E0BB27AC2DA3950E94CF2E0E94E23084
:10349000FF3A0000BB27AD2DA3950E94CF2EEBE78E
:1034A000F1E0C6EED1E0AEE141EFB191B03031F0E4
:1034B000BE8F4CAF4993AA95C1F706C0B0E2BE8F4C
:1034C0004CAF4993AA95D1F7A7E10E94B02EC0E076
:1034D000D4E0E1E1F0E10E94E1319DE050E0452FD0
:1034E0004C5FB42FAA270E94FB3015DF53955D3047
:1034F000B1F7452F4950B42FA9E00E94FB300BDFF4
:1035000053955A31B1F7A7E30E94B02EC3E1D4E03E
:10351000EDE1F0E10E94E1310E94E23004135354E6
:1035200041434B3A00009927BB27A09169010E94B3
:10353000CF2E6CE0C0916901C61720F0C61BB4E025
:10354000B60F02DF6A95B1F708954F935F936F93BB
:103550007F93EF93FF93CF93DF93AF93BF93AF929C
:10356000BF928F939F9361DEB2DD20DF2BD088273F
:10357000A0912D014D3E11F4A1600EC0413F11F408
:10358000AA270AC0423F11F4A46006C0433F71F766
:103590006BDE0E944333E9CFA0932D0140911601C9
:1035A0004030E1F761DE9F918F91BF90AF90BF9166
:1035B000AF91DF91CF91FF91EF917F916F915F91EB
:1035C0004F9108952092170162DE4091170140301B
:1035D000D9F30C94E73320922A0120923E01A5E012
:1035E0000E94B02EC0E0D0E0EDE1F6E10E947F3213
:1035F000A0E50E94B02E0E94E230010244464C41F8
:1036000053482073697A653A20000E9422204F3087
:1036100049F40E94E230FF3634204B6942797465E8
:1036200000001BC04F3749F40E94E230FF353132B1
:10363000204B69427974650010C04F3F41F40E94ED
:10364000E230FF31204D69427974650006C00E9466
:10365000E230FF302042797465000E94132041302F
:10366000B1F0C1D00E9443334D3E09F448C0443FFD
:1036700009F4B1CF413FB1F726D1ADCFECD00E94D4
:1036800043334D3E09F43BC0443FC9F7A4CF3DED61
:10369000209217010E94E7334091140144704317B0
:1036A00039F0342F403011F42FD0F4CF64D0F2CF62
:1036B00040911701403071F34D3E09F420C0509104
:1036C0001401547051F0413F19F40E94161D83CF2C
:1036D000443F11F4F8D07FCFDDCF413F11F44DD1FD
:1036E0007ACF423F19F40E946D1D75CF433F19F404
:1036F0000E94BF1D70CF443F09F46DCFCBCFA09186
:103700001601A030E1F70895A7E20E94B02E0E94B2
:10371000E23016002045786974200000A0E60E947F
:10372000B02E0E94E2301606496E666F2000A0E4BB
:103730000E94B02E0E94E230160B4261636B7570DE
:103740000000A7E10E94B02E0E94E23016115265DF
:1037500073746F726500A7E30E94B02E0E94E2307E
:103760001618526573636100AEE6A0932B07AEE6B0
:10377000A09379040895A7E20E94B02E0E94E2303F
:1037800016002020202020200000A0E60E94B02E5D
:103790000E94E230160644656C6574650000A0E482
:1037A0000E94B02E0E94E230160C20202020202003
:1037B0000000A7E10E94B02E0E94E23016122020E5
:1037C000202020200000A7E30E94B02E0E94E230BB
:1037D0001618466F726D6100AEE6A0932B07A4E742
:1037E000A09379040895A7E20E94B02E0E94E230CF
:1037F00016002045786974200000A0E60E94B02ED3
:103800000E94E2301606466F726D61740000A0E4FB
:103810000E94B02E0E94E230160C20202020202092
:103820000000A7E10E94B02E0E94E2301612202074
:10383000202020200000A7E30E94B02E0E94E2304A
:103840001618526573636100AEE6A0932B07AEE6CF
:10385000A09379040895A7E20E94B02E0E94E2305E
:1038600016002045786974200000A0E60E94B02E62
:103870000E94E23016062020202020200000A0E434
:103880000E94B02E0E94E230160C20202020202022
:103890000000A7E10E94B02E0E94E2301612202004
:1038A000202020200000A7E30E94B02E0E94E230DA
:1038B0001618526573636100AEE6A0932B07AEE65F
:1038C000A093790408950E9449374F466F726D6145
:1038D00074204D656469756D3F00413009F00895AD
:1038E000A6E20E94B02EC2E0D8E0EBE1FCE00E942C
:1038F00047320E94E2300903466F726D6174746949
:103900006E672E2E2E202020202020000E94E230E4
:103910000B0300000E942520803001F50E94E23058
:103920000903466F726D617474696E672E2E2E20C6
:10393000446F6E652100A2E70E94B02E0E94E23023
:103940000B03202020507265737320616E79206B09
:103950006579212020000E94433308950E94E230BF
:103960000903466F726D617474696E672E2E2E2086
:103970004572726F72210000DECFA0E60E94B02E69
:10398000C4E0D8E0E9E1FDE00E9447320E94E23065
:103990000905417661696C61626C653A00000E94BC
:1039A000E2300A0546696C65733A20009CE00E948B
:1039B0000520DF93CF93DF010E94CF2E0E94E230DB
:1039C000FF202F000E942220A42FB0E011960E9419
:1039D000CF2E0E94E2300B05426C6F636B733A008E
:1039E000AF91BF910E94CF2E0E94E230FF202F00A6
:1039F0000E940D20A0EFA49FD0011197B03009F4D0
:103A000013970E94CF2EA6E00E94B02E0E94E230B3
:103A10000C05202020507265737320616E79206B35
:103A20006579212020000E944333089577270AD129
:103A3000A4E00E94B02EC1E0D2E0ECE1F5E10E94EA
:103A40007F32A0E40E94B02E0E94E230030244655F
:103A50006C6574652066696C6500B0D07093580120
:103A6000D7D24C3FD1F34BD1413019F4A72F89D293
:103A7000E0D208957727E6D0A4E00E94B02EC1E0FE
:103A8000D2E0ECE1F5E10E947F32A0E40E94B02E8A
:103A9000A0E1A0935C010E94E230030253617665CD
:103AA0002050000099D28AD070935801B1D2403E84
:103AB00020F4403161F0F3D0DECFA7D2D03021F432
:103AC000CC3010F426D1D7CF5CD2B3D108950BD12E
:103AD000413089F656D2B9D108957727B3D0A4E002
:103AE0000E94B02EC1E0D2E0ECE1F5E10E947F320D
:103AF000A0E40E94B02EA2E1A0935C010E94E230FB
:103B000003024261636B7570000058D070935801D6
:103B10007FD2403920F4423161F0C1D0DFCF75D27D
:103B2000D03021F4C03610F4F4D0D8CF2AD2EED160
:103B30000895D9D0413091F624D2F4D10895772751
:103B400081D0A4E00E94B02EC1E0D2E0ECE1F5E12A
:103B50000E947F32A0E40E94B02E0E94E230030255
:103B60004C6F61642050000037D228D07093580108
:103B70004FD2403111F0A1D0E3CF87D108957727FC
:103B800061D0A4E00E94B02EC1E0D2E0ECE1F6E109
:103B90000E947F32A0E40E94B02E0E94E230030215
:103BA000526573746F72650009D07093580130D2FA
:103BB000423111F08DD0E4CFCDD10895B5D00BD1E5
:103BC0000E9443334D3E21F42FD14F914F910895E0
:103BD0004A3E09F40895403E19F40FD17727EECFFD
:103BE000413E21F40AD170916001E8CF443E49F48E
:103BF000703031F302D17150472F4F704F30F1F2D6
:103C0000DECF453E59F440916001471709F4D8CF03
:103C1000F4D07395472F4F7089F2D1CF463E29F4E7
:103C2000703170F2EAD07051C9CF473E51F44091E3
:103C300060014F3031F04051471718F0DED0705F0F
:103C4000BDCFBECF0E942220403019F44F914F913A
:103C50001BC0409360010E941A330E941A33E3D1C3
:103C6000413019F04F914F9101C008950E942037C3
:103C70004F44464C415348206E6F7420666F726DFE
:103C800061747465640008950E9420374F44464C67
:103C9000415348206572726F7221000008950E949E
:103CA00020374F43616E206E6F74207361766520FC
:103CB0006F6E20746869730008950E9420374F4E1C
:103CC0006F2042415349432066696C6500000895A6
:103CD0000E9420374F4E6F204241434B5550206683
:103CE000696C650008950E944937C04F7665727708
:103CF000726974652066696C653F000008950E94D2
:103D000049374F44656C6574652066696C653F0092
:103D100008950E9420374F4E6F20737061636520B5
:103D20006C656674000008955F936F937F93A72F6F
:103D3000A07FA0935301A0915301AF70AB5FBA2F46
:103D4000A4E00E94FB30A6E00E94B02EA091530197
:103D5000BB2795E00E94CF2E0E94A52FA5E00E94D0
:103D6000B02EA0915301A093580152D1ADD04F3F36
:103D700061F1A0915301A093580140E040935A0192
:103D800042E040935C01882757D1803091F4CCE326
:103D9000DFE00E94A52F5CE05F934991403808F076
:103DA0004EE2403208F440E20E94A62F5F915A95FD
:103DB00099F7A0915301A395A0935301AF7009F017
:103DC000BACF7F916F915F9108955DE00E94A52F1A
:103DD0005A95E1F7EECF4F935F93C4E1D5E0472FBB
:103DE0004F705EE1459FC00DD11D52EF47E15993E1
:103DF0004A95E9F75F914F9108954F935F93C4E11E
:103E0000D5E0472F4F705EE1459FC00DD11D5CE0AE
:103E100044E059934A95E9F75AE043E159934A95AA
:103E2000E9F75F914F910895A0911601A030E1F755
:103E30000895709358014CE040935A0140E140933B
:103E40005C01F4D0803009F01FCF7093580190913D
:103E50003D01E0E0F0E99770929540EC949FE00D11
:103E6000F11D40E04F9300E0CCE3DFE015911993A2
:103E70000A95E1F740935A0142E040935C01DFD09C
:103E80004F9143954C3071F7089590913D01977093
:103E9000E0E0F0E9929540EC949FE00DF11D40E0E8
:103EA0004F9340935A0142E040935C017093580154
:103EB000C3D0CCE3DFE00E94777832964F914395F0
:103EC0004C3071F778940895403139F40E94E23013
:103ED000FF4241533A0040E10895423139F40E94D3
:103EE000E230FF4255503A0042E10895443139F43E
:103EF0000E94E230FF5553523A0044E108950E9477
:103F0000E230FF2D2D2D2D004FEF089570935801B5
:103F100040E640935A0142E140935C0187D08030F3
:103F200009F0B2CE709358014427E0E0F0E94F93D6
:103F3000CCE3DFE00024159019920A94E1F7409356
:103F40005A0142E040935C017AD04F91439540364C
:103F500071F7089540E0E0E0F0E94F9340935A0193
:103F600042E040935C017093580166D0CCE3DFE0FF
:103F70000E94777832964F914395403671F7789446
:103F800008954F93FF93EF93DF93CF93BF93AF9336
:103F900040912C01409361014CE440932C01C6E018
:103FA000DAE0E7E1FCE00E9447320E94E2300B07D2
:103FB00057726974696E6720646174612E2E2E00D9
:103FC0004091610140932C01AF91BF91CF91DF915E
:103FD000EF91FF914F910895CAE2CAE240913D01ED
:103FE000942F4F5C499340E249934BE549934091AC
:103FF00029014F934068409329010E94A9784DE51B
:1040000049934F914093290108950E94B13B08952F
:104010000E947D3C0E94403A08950E94ED39089527
:104020000E946D3A08950E948C3B08950E94123CB4
:1040300008950E94853C08950E94053D08950E94C0
:10404000A63C08950E94FB3908950E941E3B0895E6
:10405000A1E00E94C53420922A0120923E01A7E0EF
:104060000E94B02EC0E0D0E0EDE1F6E10E947F3288
:10407000A0E70E94B02E0E94E23001024156522D6C
:104080004368697042617369633220636F6E666969
:10409000677061676500A7E20E94B02E0E94E2305F
:1040A00016002045786974200000A0E60E94B02E1A
:1040B0000E94E2301606204B657962200000A0E4E1
:1040C0000E94B02E0E94E230160C20536572202010
:1040D0000000A7E10E94B02E0E94E230161220508C
:1040E000617220200000AEE6A0932B07A0E2A0930F
:1040F0007904A7E30E94B02E0E94E2301618436CA8
:104100006F6E6500A7E00E94B02E0E94E23014019D
:10411000436865636B73756D3A200000D8D036D064
:104120006AD09CD00E9443334D3E09F4CBC0413F3E
:1041300061F440913C014250427040933C010E9426
:10414000007824D00E946221EDCF423F61F440917B
:104150000C014150417040930C010E9400784BD0FB
:104160000E946221DFCF433F61F440910D01415035
:10417000417040930D010E94007870D00E9462212E
:10418000D1CF443F11F40E94E52A62CFA6E00E94FD
:10419000B02E0E94E23003014B6579626F61726458
:1041A000206C61796F75743A0000A7E140913C0181
:1041B000403009F4A1E70E94B02E0E94E2300312C1
:1041C0004445202851574552545A2900A7E14091AF
:1041D0003C01423009F4A1E70E94B02E0E94E23077
:1041E0000412555320285157455254592900A7E02D
:1041F0000E94B02E0895A6E00E94B02E0E94E230E8
:10420000060153657269616C20706F72743A000028
:10421000A7E140910C01403009F4A1E70E94B02EC3
:104220000E94E2300612203132303020427073207A
:104230002000A7E140910C01413009F4A1E70E9460
:10424000B02E0E94E230071220323430302042700B
:1042500073202000A7E00E94B02E0895A6E00E94DF
:10426000B02E0E94E2300901506172616C6C656C85
:1042700020706F72743A0000A7E140910D01403048
:1042800009F4A1E70E94B02E0E94E2300912507298
:10429000696E7465722F494F2000A7E140910D01AE
:1042A000413009F4A1E70E94B02E0E94E2300A12C8
:1042B0004D656D6F72792D4578702000A7E00E94E2
:1042C000B02E0895A0911601A030E1F70895AA2715
:1042D000BB27CC27DD27EE27FF27159042E0149E51
:1042E000A00DB11DC21DD21D459147E0149EA00D29
:1042F000B11DC21DD21DF03981F7EE27F0EF4591B7
:1043000041E7149EB01DC11DD21D459147E0149E8A
:10431000B01DC11DD21DF03091F7BF93AF93DE01E8
:104320009FE00E942A2FAF91BF910E942A2F0895EB
:10433000AEE0A0932C01C1E0D4E0ECE1F1E10E94F9
:1043400047320E94E230050500000E94EF010E9402
:10435000E230060328632920323030362D38204AD7
:104360006F65726720576F6C6672616D0000A2EA1C
:10437000A0932C010E94E23008032020202020205E
:1043800044656469636174656420746F2020202033
:10439000202000000E94E2300903466C6F726961C0
:1043A0006E2C204572696B20616E64204469616ED9
:1043B000612E0000AEE0A0932C010E94E2300B02BF
:1043C0005468697320736F667477617265206973CE
:1043D000206C6963656E736564000E94E2300C04B2
:1043E000756E64657220746865207465726D7320E3
:1043F0006F662074686520000E94E2300D04474E0D
:1044000055205055424C4943204C4943454E534555
:1044100020562E3320000E94E2300E035573652093
:10442000697420617420796F7572206F776E2072C5
:1044300069736B210000A2ECA0932C010E94E23072
:10444000100720505245535320414E59204B455997
:1044500020000E944333089502414253282E2E2EFD
:104460000353474E282E2E2E04535152282E2E2E03
:10447000054E4F54282E2E2E06524E44282E2E2EF8
:1044800007414443282E2E2E08494E282E2E2E2E2C
:1044900009585045454B282E0A54454D50282E2E7C
:1044A0000B4C4F282E2E2E2E0C4849282E2E2E2E09
:1044B0000D4B4559282E2E2E0E455045454B282E86
:1044C0000F455252282E2E2E104152282E2E2E2EBF
:1044D0001153494E282E2E2E12434F53282E2E2E86
:1044E000134654595045282E144653495A45282EF0
:1044F000155053544154282E805052494E542E2E5C
:1045000081434C532E2E2E2E82474F544F2E2E2E4B
:1045100083424F582E2E2E2E8441434F50592E2E1B
:104520008553594E432E2E2E86454E442E2E2E2E2A
:104530008742434F50592E2E885448454E2E2E2EDA
:1045400089504F532E2E2E2E8A4E4F54452E2E2EEE
:104550008B454D49542E2E2E8C574B45592E2E2EC1
:104560008D524B45592E2E2E8E474F5355422E2E8F
:104570008F52455455524E2E90564D4F44452E2E37
:10458000914E4558542E2E2E92494E5055542E2E53
:1045900093504C4F542E2E2E94574149542E2E2E6C
:1045A00095545345542E2E2E96544745542E2E2E58
:1045B000974653454C454354984F4E4552522E2EE4
:1045C00099535055542E2E2E9A534745542E2E2E25
:1045D0009B45504F4B452E2E9C4745545049582ED5
:1045E0009D434952434C452E9E434F4C4F522E2ED5
:1045F0009F424F524445522EA150554D502E2E2EC3
:10460000A258504F4B452E2EA359454D49542E2E9E
:10461000A44C494D49542E2EA54745544348415278
:10462000A644524157544F2EA7504C41592E2E2E7E
:10463000A85350524954452EA95343524F4C4C2E27
:10464000AA425245414B2E2EAB464153542E2E2E9C
:10465000AC534C4F572E2E2EAD445241572E2E2E7A
:10466000AE49434F4D4D2E2EAF444154412E2E2E78
:10467000B043544558542E2EB146524541442E2E37
:10468000B24657524954452EB343424F582E2E2E10
:10469000B447455441545452B54644454C4554459D
:1046A000B646424F582E2E2EB750414C45545445D5
:1046B000B8464F522E2E2E2EB949462E2E2E2E2E75
:1046C000BA4449522E2E2E2EBB4F55542E2E2E2E2E
:1046D000BC46434952434C45BD414C4552542E2E95
:1046E000BE46435245415445BF41534B2E2E2E2EBC
:1046F000C03F2E2E2E2E2E2EC742432E2E2E2E2E75
:10470000CA4E4F2E2E2E2E2ECB454D2E2E2E2E2E19
:10471000CC574B2E2E2E2E2ECD524B2E2E2E2E2EF5
:10472000CE474F532E2E2E2ECF5245542E2E2E2EA8
:10473000C2474F2E2E2E2E2ED0564D2E2E2E2E2EE2
:10474000D2494E502E2E2E2ED3504C2E2E2E2E2EA3
:10475000D74653454C2E2E2EDC4750582E2E2E2E4B
:10476000DD43492E2E2E2E2EDE434F4C2E2E2E2E86
:10477000DF424F2E2E2E2E2EE44C494D2E2E2E2E65
:10478000E54743482E2E2E2EE644544F2E2E2E2E35
:10479000E85350522E2E2E2EED44522E2E2E2E2E1B
:1047A000EE49432E2E2E2E2EEF44412E2E2E2E2E4F
:1047B000F14652442E2E2E2EF24657522E2E2E2EDB
:1047C000F44741542E2E2E2EF54644454C2E2E2EC7
:1047D000F750414C2E2E2E2EFC4643492E2E2E2EC7
:1047E000FE4643522E2E2E2E002E2E2E2E2E2E2EF6
:1047F000A0910801B0910901ED01E2EBF2E0CE0FCA
:10480000DF1FF6E8E0910E01FE0F10900F01ED9111
:1048100049915491688160FB57FD429548B9ED91EB
:1048200056FD429548B9042E000055FD429548B901
:104830006A8153FD429548B952FD429551FD02945B
:1048400048B9549108B8499157FD429548B9ED913E
:1048500056FD429548B9042E000055FD429548B9D1
:104860006A8153FD429548B952FD429551FD02942B
:1048700048B9549108B8499157FD429548B9ED910E
:1048800056FD429548B9042E000055FD429548B9A1
:104890006A8153FD429548B952FD429551FD0294FB
:1048A00048B9549108B8499157FD429548B9ED91DE
:1048B00056FD429548B9042E000055FD429548B971
:1048C0006A8153FD429548B952FD429551FD0294CB
:1048D00048B9549108B8499157FD429548B9ED91AE
:1048E00056FD429548B9042E000055FD429548B941
:1048F0006A8153FD429548B952FD429551FD02949B
:1049000048B9549108B8499157FD429548B9ED917D
:1049100056FD429548B9042E000055FD429548B910
:104920006A8153FD429548B952FD429551FD02946A
:1049300048B9549108B8499157FD429548B9ED914D
:1049400056FD429548B9042E000055FD429548B9E0
:104950006A8153FD429548B952FD429551FD02943A
:1049600048B9549108B8499157FD429548B9ED911D
:1049700056FD429548B9042E000055FD429548B9B0
:104980006A8153FD429548B952FD429551FD02940A
:1049900048B9549108B8499157FD429548B9ED91ED
:1049A00056FD429548B9042E000055FD429548B980
:1049B0006A8153FD429548B952FD429551FD0294DA
:1049C00048B9549108B8499157FD429548B9ED91BD
:1049D00056FD429548B9042E000055FD429548B950
:1049E0006A8153FD429548B952FD429551FD0294AA
:1049F00048B9549108B8499157FD429548B9ED918D
:104A000056FD429548B9042E000055FD429548B91F
:104A10006A8153FD429548B952FD429551FD029479
:104A200048B9549108B8499157FD429548B9ED915C
:104A300056FD429548B9042E000055FD429548B9EF
:104A40006A8153FD429548B952FD429551FD029449
:104A500048B9549108B8499157FD429548B9ED912C
:104A600056FD429548B9042E000055FD429548B9BF
:104A70006A8153FD429548B952FD429551FD029419
:104A800048B9549108B8499157FD429548B9ED91FC
:104A900056FD429548B9042E000055FD429548B98F
:104AA0006A8153FD429548B952FD429551FD0294E9
:104AB00048B9549108B8499157FD429548B9ED91CC
:104AC00056FD429548B9042E000055FD429548B95F
:104AD0006A8153FD429548B952FD429551FD0294B9
:104AE00048B9549108B8499157FD429548B9ED919C
:104AF00056FD429548B9042E000055FD429548B92F
:104B00006A8153FD429548B952FD429551FD029488
:104B100048B9549108B8499157FD429548B9ED916B
:104B200056FD429548B9042E000055FD429548B9FE
:104B30006A8153FD429548B952FD429551FD029458
:104B400048B9549108B8499157FD429548B9ED913B
:104B500056FD429548B9042E000055FD429548B9CE
:104B60006A8153FD429548B952FD429551FD029428
:104B700048B9549108B8499157FD429548B9ED910B
:104B800056FD429548B9042E000055FD429548B99E
:104B90006A8153FD429548B952FD429551FD0294F8
:104BA00048B9549108B8499157FD429548B9ED91DB
:104BB00056FD429548B9042E000055FD429548B96E
:104BC0006A8153FD429548B952FD429551FD0294C8
:104BD00048B9549108B8499157FD429548B9ED91AB
:104BE00056FD429548B9042E000055FD429548B93E
:104BF0006A8153FD429548B952FD429551FD029498
:104C000048B9549108B8499157FD429548B9ED917A
:104C100056FD429548B9042E000055FD429548B90D
:104C20006A8153FD429548B952FD429551FD029467
:104C300048B9549108B8499157FD429548B9ED914A
:104C400056FD429548B9042E000055FD429548B9DD
:104C50006A8153FD429548B952FD429551FD029437
:104C600048B9549108B8499157FD429548B9ED911A
:104C700056FD429548B9042E000055FD429548B9AD
:104C80006A8153FD429548B952FD429551FD029407
:104C900048B9549108B8499157FD429548B9ED91EA
:104CA00056FD429548B9042E000055FD429548B97D
:104CB0006A8153FD429548B952FD429551FD0294D7
:104CC00048B9549108B8499157FD429548B9ED91BA
:104CD00056FD429548B9042E000055FD429548B94D
:104CE0006A8153FD429548B952FD429551FD0294A7
:104CF00048B9549108B8499157FD429548B9ED918A
:104D000056FD429548B9042E000055FD429548B91C
:104D10006A8153FD429548B952FD429551FD029476
:104D200048B9549108B8499157FD429548B9ED9159
:104D300056FD429548B9042E000055FD429548B9EC
:104D40006A8153FD429548B952FD429551FD029446
:104D500048B9549108B8499157FD429548B9ED9129
:104D600056FD429548B9042E000055FD429548B9BC
:104D70006A8153FD429548B952FD429551FD029416
:104D800048B9549108B8499157FD429548B9ED91F9
:104D900056FD429548B9042E000055FD429548B98C
:104DA0006A8153FD429548B952FD429551FD0294E6
:104DB00048B9549108B8499157FD429518B8EE91F9
:104DC000F0910E01F395FA3029F4FF27A093080122
:104DD000B0930901F0930E010C94182DA0910801D5
:104DE000B0910901C0914101D82DF6EFE0910E017B
:104DF000FE0FE395E0930E01EA3088F1EC3069F59F
:104E00009396A0930801B093090120920E01DC3023
:104E100031F4C0914001C09341010C94182DD83158
:104E200089F4A1E3B2E0C0912E01D3E2CD9FA00DA1
:104E3000B11DCEE0A0930801B0930901C0934101D8
:104E40000C94182DD83D49F4C4EEAEE0B2E0A09326
:104E50000801B0930901C09341010C94182DCF9221
:104E6000DF92EF92FF92D83D50F4CC2EDC2EEC2E48
:104E7000FC2E0000000000000000000009C0CEE68B
:104E8000FC2ECEE2EC2EC0E8DC2EC0ECCC2ECEE424
:104E900010900F01ED9154914C2F57FD429548B958
:104EA00056FD4295042E48B955FD02944C2F08B882
:104EB00053FD029408B852FD0294000008B8ED9129
:104EC00048B9549157FD429548B956FD4295042E74
:104ED00048B955FD02944C2F08B853FD029408B808
:104EE00052FD0294000008B8ED9148B9549157FD65
:104EF000429548B956FD4295042E48B955FD029495
:104F00004C2F08B853FD029408B852FD02940000DB
:104F100008B8ED9148B9549157FD429548B956FDEE
:104F20004295042E48B955FD02944C2F08B853FD04
:104F3000029408B852FD0294000008B8ED9148B9F7
:104F4000549157FD429548B956FD4295042E48B9F3
:104F500055FD02944C2F08B853FD029408B852FD39
:104F60000294000008B8ED9148B9549157FD42955C
:104F700048B956FD4295042E48B955FD02944C2F70
:104F800008B853FD029408B852FD0294000008B816
:104F9000ED9148B9549157FD429548B956FD429557
:104FA000042E48B955FD02944C2D08B853FD0294C7
:104FB00008B852FD0294000008B8ED9148B9549128
:104FC00057FD429548B956FD4295042E48B955FD06
:104FD00002944C2D08B853FD029408B852FD029477
:104FE000000008B8ED9148B9549157FD429548B971
:104FF00056FD4295042E48B955FD02944C2D08B833
:1050000053FD029408B852FD0294000008B8ED91D7
:1050100048B9549157FD429548B956FD4295042E22
:1050200048B955FD02944C2D08B853FD029408B8B8
:1050300052FD0294000008B8ED9148B9549157FD13
:10504000429548B956FD4295042E48B955FD029443
:105050004C2D08B853FD029408B852FD029400008C
:1050600008B8ED9148B9549157FD429548B956FD9D
:105070004295042E48B955FD02944C2D08B853FDB5
:10508000029408B852FD0294000008B8ED9148B9A6
:10509000549157FD429548B956FD4295042E48B9A2
:1050A00055FD02944C2D08B853FD029408B852FDEA
:1050B0000294000008B8ED9148B9549157FD42950B
:1050C00048B956FD4295042E48B955FD02944D2D20
:1050D00008B853FD029408B852FD0294000008B8C5
:1050E000ED9148B9549157FD429548B956FD429506
:1050F000042E48B955FD02944D2D08B853FD029475
:1051000008B852FD0294000008B8ED9148B95491D6
:1051100057FD429548B956FD4295042E48B955FDB4
:1051200002944D2D08B853FD029408B852FD029424
:10513000000008B8ED9148B9549157FD429548B91F
:1051400056FD4295042E48B955FD02944D2D08B8E0
:1051500053FD029408B852FD0294000008B8ED9186
:1051600048B9549157FD429548B956FD4295042ED1
:1051700048B955FD02944D2D08B853FD029408B866
:1051800052FD0294000008B8ED9148B9549157FDC2
:10519000429548B956FD4295042E48B955FD0294F2
:1051A0004D2D08B853FD029408B852FD029400003A
:1051B00008B8ED9148B9549157FD429548B956FD4C
:1051C0004295042E48B955FD02944D2D08B853FD63
:1051D000029408B852FD0294000008B8ED9148B955
:1051E000549157FD429548B956FD4295042E48B951
:1051F00055FD02944E2D08B853FD029408B852FD97
:105200000294000008B8ED9148B9549157FD4295B9
:1052100048B956FD4295042E48B955FD02944E2DCD
:1052200008B853FD029408B852FD0294000008B873
:10523000ED9148B9549157FD429548B956FD4295B4
:10524000042E48B955FD02944E2D08B853FD029422
:1052500008B852FD0294000008B8ED9148B9549185
:1052600057FD429548B956FD4295042E48B955FD63
:1052700002944E2D08B853FD029408B852FD0294D2
:10528000000008B8ED9148B9549157FD429548B9CE
:1052900056FD4295042E48B955FD02944E2D08B88E
:1052A00053FD029408B852FD0294000008B8ED9135
:1052B00048B9549157FD429548B956FD4295042E80
:1052C00048B955FD02944E2D08B853FD029408B814
:1052D00052FD0294000008B8ED9148B9549157FD71
:1052E000429548B956FD4295042E48B955FD0294A1
:1052F0004E2D08B853FD029408B852FD02940000E8
:1053000008B8ED9148B9549157FD429548B956FDFA
:105310004295042E48B955FD02944F2D08B853FD0F
:10532000029408B852FD0294000008B8ED9148B903
:10533000549157FD429548B956FD4295042E48B9FF
:1053400055FD02944F2D08B853FD029408B852FD44
:105350000294000008B8ED9148B9549157FD429568
:1053600048B956FD4295042E48B955FD02944F2D7B
:1053700008B853FD029408B852FD0294000008B822
:10538000ED9148B9549157FD429548B956FD429563
:10539000042E48B955FD02944F2D08B853FD0294D0
:1053A00008B852FD0294000008B8ED9148B9549134
:1053B00057FD429548B956FD4295042E48B955FD12
:1053C00002944F2D08B853FD029408B852FD029480
:1053D000000008B8ED9148B9549157FD429548B97D
:1053E00056FD4295042E48B955FD02944F2D08B83C
:1053F00053FD029408B852FD0294000008B8ED91E4
:1054000048B9549157FD429548B956FD4295042E2E
:1054100048B955FD02944F2D08B853FD029408B8C1
:1054200052FD0294000008B8ED9148B9549157FD1F
:10543000429548B956FD4295042E48B955FD02944F
:105440004F2D08B853FD029408B852FD0294000095
:1054500008B8ED9148B9549157FD429518B8FF909E
:10546000EF90DF90CF900C94182DA0910801B0918F
:105470000901D0910001C0910101C295DC0FDE7ECF
:10548000E5E110900F01FD914D2FF0FD429548B9D7
:1054900000004D2FF1FD429548B900004D2FF2FD5F
:1054A000429548B900004D2FF3FD4295000048B9E0
:1054B0006D2F4D2FF4FD429548B9CD91F5FD6295C4
:1054C0005D2F68B9F6FD52956D2F4D2F58B9F7FD38
:1054D0006295C0FD4295000068B9FC2FEA95B9F6C7
:1054E00018B8EE91F0910E01F395F23029F4FF27F0
:1054F000A0930801B0930901F0930E010C94182DAC
:10550000A0910801B0910901D1E0FEE110900F01D6
:10551000ED91CE2FC370588158B9CE2FC695C69540
:10552000C3705881E29558B9CE2FC3705881CE2FE1
:10553000C69558B9C695C3705881ED91CE2F58B90C
:10554000C3705881FA9541F718B8EE91F0910E01A9
:10555000F395F33029F4FF27A0930801B0930901D4
:10556000F0930E010C94182DA0910801B09109013F
:105570000F9310900F01EAE2D1E0CD91C6950C2F68
:10558000C295C770F881F8B9C02F0000C770F881C4
:10559000000000000000F8B9CD91C6950C2FC2950F
:1055A000C770F881EA9579F718B811970F91F091C3
:1055B0000E01F395F43029F4FF27A0930801B0936E
:1055C0000901F0930E010C94182D0E9449376F4386
:1055D0006C6F6E652073797374656D3F2000413088
:1055E00009F0089565D087D0803079F078D00E9496
:1055F00020374F4E6F20636F6E74726F6C6C6572E4
:1056000020666F756E64200008958DD0803069F03B
:1056100066D00E9420374F4E6F204D65676136344B
:105620003420666F756E64000895CBD09BD0EE2752
:10563000FF2750E060E00590B6D00590BBD06395A1
:105640006038C9F79CD05395A9F74CEA4ED040EA90
:105650004CD04AD046EE49D00E941A330E941A33E9
:105660000E941A334CEA41D048EA3FD03DD041ED88
:105670003CD00E941A330E941A330E941A334CEA1B
:1056800034D044EA32D030D04CEF2FD00E941A33BD
:105690000E941A330E941A3322D00E94203780536E
:1056A000797374656D20636C6F6E65640000089596
:1056B00043E54CBD2DBC249A2C984FEF4A95F1F749
:1056C0002C9A4FEF4A95F1F72C984FEF4A95F1F746
:1056D0002C984FEF4A95F1F70E941A3308952C9AAF
:1056E0004CE54CBD3DBC089544274EBD4DB547FF2C
:1056F000FDCF4EB5089588274CEAF7DF43E5F5DF87
:10570000F3DF433509F081E0EFDF0895BF93AF93F6
:105710004F93A42FBB270E942A2F0E94A52F4F91A1
:10572000AF91BF910895882740E3DFDFDDDF40E0E0
:10573000DCDFDADF4E3111F082E0089540E3D5DF9F
:10574000D3DF41E0D2DFD0DF463911F082E00895A7
:1057500040E3CBDFC9DF42E0C8DFC6DF493009F0F4
:1057600082E008954CEAC1DF40E8BFDFBDDFBCDF67
:105770000E941A330E941A330E941A3308954CE48F
:10578000B4DF452F4695B1DF452F440F440F440F3A
:10579000440F440F440F440FA8DFA6DF0E941A33C2
:1057A0000E941A33089540E4A0DF9EDF462F9DDF5C
:1057B000402D9BCF48E499DF97DF462F96DF402DA1
:1057C00094CF4F93FF93EF93DF93CF93BF93AF9318
:1057D00040912C01409361014CE440932C01C5E0C1
:1057E000DAE0E8E1FCE00E9447320E94E2300B067A
:1057F000436C6F6E696E672053797374656D2E2EDE
:105800002E004091610140932C01AF91BF91CF9147
:10581000DF91EF91FF914F91089528B818954F931C
:105820005F936F93FF93EF93DF93CF93BF93AF9308
:105830000F921F92FFB7FF9330921101B091310187
:10584000B7FF5C98B7FD5C9A4B99BE7F4B9BB160EC
:10585000B0933101C8E0D1E05F89A889E9890A885D
:105860001B88A00DE11DA88BE98BFFA14491AD8998
:10587000AF3F09F0452F5AA54503B0E8B10DB093ED
:10588000B300EE89FF89488D598DAA27E2FDA095C6
:10589000E5FDA095F4FDA09557FDA095AA1FEE1F6C
:1058A000FF1F441F551FEE8BFF8B488F598F830CB2
:1058B000921CEBA9FF81EF23E8B97894E9A190FC51
:1058C00004C0F8A58F1608F490C0FCE0E2FFFDEEDE
:1058D0008F1639F45E98E3FFABC0B2E8B093800056
:1058E000A7C0F1E1E2FFF3EF8F1639F45E9AE3FF10
:1058F0009FC0B2ECB09380009BC0FBE1E2FFFFEFE2
:105900008F1621F4EFEFE0933B0192C0F2E0E2FF4B
:10591000F9EE8F1619F420923B018AC0F9E3E2FFF9
:10592000F7E08F1609F084C0A8ECA883A1E0A98352
:105930002E8288249924AAE0A9AFA5E0E2FFA395CE
:1059400042E3E2FF4CE3BA8DB395BA1731F4BB27BB
:10595000EB8DFC8D3196EB8FFC8FBA8FE885E3954C
:10596000E41709F4EE27E887F5E8E0E0AC89EA0FF0
:10597000F21DB491B21511F0A395AC8BBAA7A0910A
:105980005001A03009F454C0B0915101B395B093C7
:105990005101BA17C0F3BB27B0935101E0915201F6
:1059A000F0915301C0915601D09157012196A191D8
:1059B000E0935201F0935301AE3F09F044D6FD1736
:1059C00098F0EC1788F0A0913301A13029F4A2E0FF
:1059D00020925001A0933301E0915401F0915501C0
:1059E000E0935201F093530123C0A0918400AA3F99
:1059F000E0F3AB3F00F0AC3F00F0AD3F00F0AE3F56
:105A000000F0E5FD15C0E0912901E7FD0C94EE26BC
:105A1000E0913E01E37011F40C94F823E13011F4AD
:105A20000C94352AE23011F40C94802A0C94B42A98
:105A3000A0911401A5FD22C0E091C000E7FF64C061
:105A4000E091C600F2E8B491B0FF33C0A7FF03C0F5
:105A50002092160156C0E33809F4E0E1FEE74091D8
:105A60003C01F40FEF77A4FFA6FDF395A4FFA0FD82
:105A7000E068E491E0931501A06244C0E091150153
:105A8000E0931601E0931701EE3E19F4A2FD0C9489
:105A9000380040912D01E33611F4A2FD4160E0375A
:105AA00011F4A2FD4260EC3F09F4446040932D01E3
:105AB00028C0E03F11F4A06825C0E03E11F4A064C6
:105AC00021C0E23121F4A160A7FDAE7F1AC0E93503
:105AD00021F4A260A7FDAD7F14C0E43151F4A6FD0E
:105AE00004C0A460A7FDAB7F0CC0A860A7FDA77F82
:105AF00008C0E13121F4A061A7FDAF7E02C0209271
:105B00001601AF71A093140140910C0140FD31C00A
:105B1000A0913101E0912701E03091F0EF3F21F4B5
:105B2000A0FD0EC0ECE70CC0EA95F2E8B491B7FF17
:105B300007C0B0912801B695A0FBB7F9B093280132
:105B4000E0932701E0912501E03091F0EF3F19F457
:105B5000E0E9AF770DC0EA95F2E8B491B6FF08C06E
:105B6000B0912601B0FB0894B795A7F9B093260130
:105B700030C0A0913101E0912701E03091F0EF3F7A
:105B800021F4A0FD0EC0EEE30CC0EA95F2E8B4915A
:105B9000B5FF07C0B0912801B695A0FBB7F9B09347
:105BA0002801E0932701E0912501E03091F0EF3FDB
:105BB00019F4E8E4AF770DC0EA95F2E8B491B4FFC8
:105BC00008C0B0912601B0FB0894B795A7F9B0932F
:105BD0002601E0932501A0933101FF91FFBF1F90A3
:105BE0000F90AF91BF91CF91DF91EF91FF916F91A6
:105BF0005F914F911895AAEBA4B9AFEFA5B9A0EEAC
:105C0000A7B9A0E0A8B9A0EFAAB9AFEFABB9A6B108
:105C1000AF77A0932901B2ECB0938000B9E1B093C3
:105C20008100F4E0A2FFF4E0F0938700FEEFA2FF12
:105C3000F6EFF093860020928900FAE5F093880051
:105C4000F4E0F0938B00F8EDF0938A00A6E0A093C7
:105C50006F00A2E0A4BDA1E0A5BDA1E3A7BDA3E89C
:105C6000A093B000A1E0A093B100A0E8A093B3007E
:105C70002092B6002092C000A0E1A093C100A6E649
:105C8000A093C200ACE5ACBDA1E0ADBDA5E168D07C
:105C9000C8E0D1E0A8ECA993A1E0A993AEE12992D4
:105CA000AA95E9F7AAEAA0931E01A09320012092E9
:105CB0002A01AEE3A0931C010F93009129010F77F5
:105CC0000093290106EE07C00F9300912901006897
:105CD0000093290104EE009330010F910895A093E1
:105CE0003E01A03041F4ACE3A0934401AEE2A093A6
:105CF0004501A6EE32C0A13069F4A8EAA0934401A0
:105D0000A4E7A0934501A0E0A0930001A0EEA0931A
:105D1000010122C0A23091F4A8E7A0934401ACE4B1
:105D2000A0934501C0E0D1E0A0E0A993A0E4A9932D
:105D3000A0EAA993A0EEA993A3EE0FC0A4E5A093B7
:105D40004401AAE3A0934501C0E0D1E0AA27B8E04E
:105D5000A993A05EBA95E1F7A7EEA09330018FC09A
:105D6000AA0FAE7EA0932C010895A295AA0FA07E43
:105D7000A0930F01089548834091290147FD0EC06B
:105D8000CF93DF935F9342EBC40F42E0D41F409167
:105D90002C014E7E48835F91DF91CF9108954F9300
:105DA0005F936F93AF93BF9340E2592F537052307C
:105DB00061F0533009F44BE2B7FF05C0A095B095F0
:105DC000A30DB21D4DE20E94A62F592F5C70692FC2
:105DD0006073E8944FE24395A051B742E0F7A05FAB
:105DE000B84D5C3009F42BD04FE24395A85EB34028
:105DF000E0F7A851BC4F53FD22D0603309F4A3D083
:105E00004FE24395A456B209E0F7AC59BF4F50306A
:105E100009F015D0603209F496D04FE24395AA50AC
:105E2000E8F70DD0A65F603109F48DD040E34A0F4A
:105E30008DD0BF91AF916F915F914F910895403395
:105E400011F0689483C091FD81C0F6F390FF08952E
:105E50007CC008954F9390FF05C04B2F429509D009
:105E60004B2F07D04A2F429504D04A2F02D04F9192
:105E700008954F70405D4A3308F0495F67C0409114
:105E80003E014030B1F0AF93BF93CF93DF93D1E0A9
:105E9000C8ECACE5BEE12992BA95E9F7AA95D1F72D
:105EA000DF91CF91AA24BB2420922B01BF91AF9107
:105EB0000895AF93BF93CF93DF93D1E0C8ECA7E1F0
:105EC000BEE14993BA95E9F7AA95D1F740912C0123
:105ED0004E7EA7E1BEE14993BA95E9F7AA95D1F7BD
:105EE000DF91CF91AA24BB2420922B01BF91AF91C7
:105EF0000895AF93BF9320922B01A0912A01A03067
:105F000051F4A7E1AA24B394AB1571F7B6E1BB2E07
:105F1000CF93DF9362C0A13029F4BF91AF914AE0E3
:105F20000C94CD34A23021F4BF91AF914AE038C433
:105F3000A33019F4BF91AF910895BF91AF915AE08A
:105F40000E94283908954CE201C040E2AF93BF930C
:105F5000A0912B01A395A0932B01A0912A01A4301D
:105F600030F0BF91AF91542F0E9428390895A0308E
:105F7000A9F0A33059F4A42FBB275F936F930E941D
:105F8000E4166F915F91BF91AF910895BF91AF916A
:105F9000A0912A01A1FF0C94CD3402C4EF93E091AB
:105FA0003E01E03009F09EC0EF91CF93DF93D7D34D
:105FB00096FD35C0E0DEA395AE3131F4AA27B39546
:105FC000B73111F4B6E107C0AA2EBB2EDF91CF91F5
:105FD000BF91AF910895AA2EBB2ED1E0C8EC4F938C
:105FE000A6E1BEE14E8D4993BA95E1F7AA95C9F7AE
:105FF000AEE140E24993AA95E9F7D4E0CAE7A6E109
:10600000BEE14E8D4993BA95E1F7AA95C9F7AEE185
:1060100040912C014993AA95E9F74F91D7CFAB3125
:10602000A8F6B23198F6AD5FAA2EEF93FF934F9288
:106030005F926F927F9270F85F93E42FF6E8B5E07D
:106040004424552466245527A491A7FD539550FB5D
:1060500040F8A6FD53955F9350FB41F8A5FD53957D
:1060600050FB50F8A3FD539550FB51F8A2FD5395FA
:1060700050FB60F85F91A1FD539550FB61F8F395DB
:106080005527A491A7FD539550FB42F8A6FD5395C3
:106090005F9350FB43F8A5FD539550FB52F8A3FDC9
:1060A000539550FB53F8A2FD539550FB62F85F9156
:1060B000A1FD539550FB63F8F395442D5CDE2196CA
:1060C000452D59DE2196462D56DE6C96BA9509F07F
:1060D000B7CF5F9170FA7F906F905F904F90FF9174
:1060E000EF9174CFFF93CF93DF936F93E42FF6E894
:1060F000AA2DBB2DDAE0C49117D0B395AA2D96FD39
:1061000013D096FDB395F395AA2DDA95A1F7AA2D94
:10611000AA5F96FDAA5FAA2E6F91DF91CF91FF91A2
:10612000EF91BF91AF91089560912C016F936295AB
:10613000C7FD629560932C0171D0A39596FD6ED03A
:1061400096FDA395C6FD62956F9360932C0166D072
:10615000A39596FD63D096FDA395C5FD62956093CA
:106160002C015CD0A39596FD59D096FDA395C3FD57
:10617000629560932C0152D0A39596FD4FD096FD69
:10618000A395C2FD629560932C0148D0A39596FD1E
:1061900045D096FDA3956F91C1FD629560932C014A
:1061A0003DD0A39596FD3AD096FDA3956F9160934F
:1061B0002C0108954F934591403011F44F9108956B
:1061C000C5DEF9CFFF91EF91EE0FFF1FAF93BF93A5
:1061D000B591BF3F11F0A5910ED0BF91AF914F93F4
:1061E0004591403031F44F913197F695E7953196CE
:1061F0000994ACDEF5CFEF93E0913E01E03021F061
:10620000EF91AA2EBB2E0895EF91AE3108F0ADE1CB
:10621000B73108F0B6E1AA2EBB2E0895CF93DF93D5
:10622000C0914401CA1728F0C0914501CB1708F06E
:1062300003C0DF91CF910895AF93BF934F935F93C6
:10624000C0913E01C37031F0C23008F441C009F47E
:1062500060C07DC051E0AC3360F5BE3250F5B0FD9A
:10626000550FB0FD550FA0FD550FB695A695CEE183
:10627000BC9FD1E0C8ECCA0FD21DC00DD11DA2EB4E
:10628000B2E0CA0FDB1FA881B0912C01BE70B2959D
:10629000A07EBA17A9F0B0912C01BE70AB2BAE7ED8
:1062A000A883A2EBB2E0CA1BDB0BB881B52BBF7091
:1062B000B8835F914F91BF91AF91DF91CF910895D6
:1062C000A2EBB2E0CA1BDB0BB8815095B523EFCF30
:1062D000CA2FC770C39540E00894441FCA95E9F7D8
:1062E000A695A695A695C5E1BC9FD1E0C8ECCA0FBE
:1062F000D21DC00DD11DA0912C01A695A17029F42D
:106300004095A881A423A883D4CFA881A42BA883D7
:10631000D0CFCA2F50912C015695537043E0C370D3
:1063200031F0440F440F550F550FCA95C9F74095EA
:10633000A695A695CEE1BC9FD1E0C8ECCA0FD21DB0
:10634000C00DD11DA881A423A52BA883B2CFCA2F2D
:1063500050912C015E704EE0C17011F4429552953F
:106360004095A695CAE2BC9FD1E0C8ECCA0FD21DE9
:10637000C00DD11DA881A423A52BA8839ACFCE310F
:1063800008F0CDE1EE3108F0EDE1D73108F0D6E1CB
:10639000F73108F0F6E1EC1718F40E2EEC2FC02DB3
:1063A000FD1718F40F2EFD2FD02D0895EC1718F4BB
:1063B0000E2EEC2FC02DFD1718F40F2EFD2FD02D13
:1063C0000895AF93BF93CF93DF93EF93FF935F93C2
:1063D000D6DFAC2FBD2FCF93DF93C3D1288252EBF2
:1063E000C50F52E0D51F50912C015883DF91CF91FA
:1063F000AE1711F0A395EFCFBF1719F0AC2FB395DF
:10640000EACF5F91FF91EF91DF91CF91BF91AF9173
:106410000895AF93BF93CF93DF93EF93FF935F9371
:10642000C5DFAC2FBD2FFADEA395AE17E1F7F6DE80
:10643000B395FB17E1F7F2DEAA95AC17E1F7EEDEB4
:10644000BA95BD17E1F75F91FF91EF91DF91CF9181
:10645000BF91AF910895AF93BF93CF93DF93EF9325
:10646000FF935F93A3DFBD2FAC2FD8DEAE1711F0E3
:10647000A395FBCFD3DEFB1711F0B395F5CF5F915A
:10648000FF91EF91DF91CF91BF91AF91089599DF87
:10649000AF93BF93CF93DF93EF93FF934F935F93AC
:1064A0006EDF4C2FBD2FAC2F5CD152EF599351EFC3
:1064B000A395AE1711F05993FBCF53EF5993A42F27
:1064C000B395BF1739F04DD150EF5993AE2F49D145
:1064D0005993F5CFA42F45D154EF599351EFA3957C
:1064E000AE1711F05993FBCF55EF59935F914F9130
:1064F000FF91EF91DF91CF91BF91AF910895C7DFE9
:106500005F93AF93BF93CF93DF93EF93FF9337DF07
:10651000BD2FAC2F26D15BEF59935CEEA395AE1740
:1065200011F05993FBCF5CEF5993FF91EF91DF91FD
:10653000CF91CF93DF93EF93FF93BD2FAC2FB39504
:1065400010D15DEF599350E2A395AE1711F0599316
:10655000FBCF5EEF5993FF91EF91DF91CF91CF93F6
:10656000DF93EF93FF93BD2FAC2FB395AF93F9D08B
:10657000A2EBB2E0CA0FDB1F50912C0152955E7E58
:106580002196AF91A395AE1711F05993FBCFFF91D0
:10659000EF91DF91CF91CF93DF93EF93FF93BD2FD7
:1065A000AC2FBE5FDED05EEE59935DEEA395AE17C5
:1065B00011F05993FBCF5FEE5993FF91EF91DF916B
:1065C000CF91BF91AF915F9108950F931F932F9338
:1065D0003F93AF93BF93CF93DF93DE010FEFCE1BBB
:1065E00010F40195C1951FEFDF1B10F41195D195A3
:1065F000CD1760F000C02C2F269510DEAE1789F065
:10660000A00F2D1BD0F7B10F2C0FF7CF2D2F2695F4
:1066100005DEBF1731F0B10F2C1BD0F7A00F2D0FE7
:10662000F7CFDF91CF91BF91AF913F912F911F9104
:106630000F910895AF93A82DA73EE9F3A82DA73E8B
:10664000E9F7AF910895EF93FF93AF93A0931D01E6
:10665000F3E8A6FDF4E8F0932F01AF73AA0FF5E875
:10666000E0E8EA0FF21DA591A0931A01A591A0936D
:106670001B0120921C012092180120921901AF9158
:10668000FF91EF910895209217014091170140303A
:10669000E1F39DC0409116014030E1F708955FD0CD
:1066A000A2EBCA0FA2E0DA1FA881BA2FAF93A171A3
:1066B000BE7EB295BA2BAF9120921701409117017F
:1066C000403041F4409110014B3110F4A883F6CFD3
:1066D000B883F4CFA8837BD042C03F933DED52D026
:1066E00020921701409114014470431749F0403043
:1066F00021F40E94F206342F03C00E941807342FA1
:1067000040911701403061F4409110014B3120F469
:1067100048814F774883E6CF488140684883E2CF7D
:1067200058815F7758833F910895D1E0C3EDCA0F38
:10673000D21D2092170140911701403061F4409121
:1067400010014B3120F448814F774883F4CF4881C2
:1067500040684883F0CF58815F7758830895AA2D09
:10676000BB2DDEE1BD9FD1E0C8ECCA0FD21DC00D2C
:10677000D11D0895F6DF0F9302EBC00F02E0D01F8A
:106780000F910895D3E2BD9FD2E0C4E3CA0FD21D9A
:10679000C00DD11D0895AA2DBB2DAA95B3952BCD63
:1067A000BF93B0910D01B0FD0EC0BFEFB1B90000B5
:1067B0001A99FECF42B9B4E6BA95F1F72998B4E632
:1067C000BA95F1F7299ABF9108954F9108954F9383
:1067D00040912D0141FFF9CF4D7F40932D01FF9353
:1067E000EF93DF93CF9340913E01403029F44091E5
:1067F000290147FF10C02CC04F9347E4CED04F91E2
:106800004F93405DCAD04F91413009F457C0423098
:1068100009F473C097C044E50E94CD344AE00E9459
:10682000CD34C8ECD1E0FEE2EEE148814295A6D03D
:106830004991A4D0EA95C9F74AE00E94CD34FA956F
:1068400099F7CF91DF91EF91FF914F9144270895F0
:1068500045E40E94CD34409140018DD04AE00E9431
:10686000CD34C8ECD1E0F3E0E3E24881429586D034
:10687000499184D0EA95C9F74AE00E94CD34FA954F
:1068800099F7E3E2F0912E01EF9FC00DD11DF0E1E9
:10689000E3E248814F77429571D049914F776ED0AE
:1068A000EA95B9F74AE00E94CD34FA9589F7CF917D
:1068B000DF91EF91FF914F9144270895409100019E
:1068C0005AD04091010157D04AE067D0C8ECD1E0DE
:1068D000F4E7E5E14881429551D049914FD0EA95DE
:1068E000C9F74AE00E94CD34FA9599F7CF91DF912C
:1068F000EF91FF914F9144270895409100013BD0C3
:106900004091010138D04091020135D040910301FE
:1069100032D04AE042D0C8ECD1E0F4E5EEE1488163
:1069200042952CD049912AD0EA95C9F74AE00E94B5
:10693000CD34FA9599F7CF91DF91EF91FF914F9177
:10694000442708954AE029D0C8ECD1E0FAE3EAE20E
:106950004881429513D0499111D0EA95C9F74AE090
:106960000E94CD34FA9599F7CF91DF91EF91FF9185
:106970004F91442708954295469547704F70405D6A
:106980004A3308F0495F0C94CD34BF93B2E0A03095
:1069900009F0B064B4BDBF910895BF93B0912501D3
:1069A000B030E1F740932601BA95B0932501BF912D
:1069B0000895BF93B0912701B030E1F7BA95B09335
:1069C0002701B0912701B030E1F740912801BF9134
:1069D0000895BF93B0912701B030E1F7BA95B09315
:1069E0002701409116014D3E41F0B0912701B03092
:1069F000C1F740912801BF9108954BE1BF910895DF
:106A0000FF93EF930F93E0911E01A0911F01B091AE
:106A10002001F09121010027E2FD0095E5FD0095A0
:106A2000A4FD0095F7FD0095001FEE1FAA1FBB1FD8
:106A3000FF1FE0931E01A0931F01B0932001F0936C
:106A400021010F91EF91FF910895FF93EF93DF9351
:106A5000CF93BF93AF934F935F936F937F934F9277
:106A60005F926F927F9240904601509049016090F2
:106A7000480170904B015091470160914A01A091EB
:106A80003E01E52F660FEE0FA33031F0660FEE0FDB
:106A9000A23011F0660FEE0FF62FA0914C01A1303D
:106AA00071F4E20146D0803011F08FE133C0E30190
:106AB00040D0803011F080E22DC065D02BC0A230D4
:106AC00091F4E20136D0803011F08FE123C0E30170
:106AD0003FD0803011F082E11DC0ACE3BDE06A0E12
:106AE0007B1E75D017C0A33011F085E113C0A52D12
:106AF000A33010F082E10EC0ACE3BDE04A0E5B1E95
:106B0000F20151916191E30114D0803011F080E2E3
:106B100001C067D07F906F905F904F907F916F9191
:106B20005F914F91AF91BF91CF91DF91EF91FF9125
:106B30000895CE0F10F48FE10895A0914401CA1773
:106B4000D0F7DF0FC0F3B0914501DB17A0F7089530
:106B5000659FC00DD11D2296D33008F082E10895C3
:106B6000A0913E015091470160914A01E52F660FC7
:106B7000EE0FA33031F0660FEE0FA23011F0660F6A
:106B8000EE0FF62F0895571478F0D20134D0E0E8D4
:106B9000FBE062D0D3012FD0E0E8FBE08AD0539431
:106BA00073946A9591F70895560E760E5A947A94D6
:106BB000D20121D0E0E8FBE04FD0D3011CD0E0E8C7
:106BC000FBE077D05A947A946A9591F70895F3018F
:106BD00051936193D2010FD03FD053946A95D1F76E
:106BE0000895F20151916191D30105D062D073945F
:106BF0006A95D1F708956F93C8ECD1E060913E019A
:106C0000613069F465E1B69FC00DD11D6A2F6695AC
:106C100066956695C60FD21D4A2F6F910895623012
:106C200069F46EE1B69FC00DD11D6A2F6695669519
:106C3000C60FD21D4A2F440F6F9108956AE2B69F86
:106C4000C00DD11D6A2F66956695C60FD21D4A2FBD
:106C5000440F440F6F9108957F936F93BF93AF9349
:106C6000652F742F777049F4A991A1936A95E1F784
:106C7000AF91BF916F917F910895B0E8713019F095
:106C8000B6957A95FBCF7727A991AB9F703019F015
:106C9000A291A029A193119273957617A9F7A991B2
:106CA000AB9FA291A029A193AF91BF916F917F91CA
:106CB00008957F936F93BF93AF93652F742F777071
:106CC00049F4A191A9936A95E1F7AF91BF916F91B2
:106CD0007F9108950F931F930FEF11E0000F110F95
:106CE0007A95E1F7652F7881009570230095A19141
:106CF000A19F072A0992712D6A95C9F768816023BF
:106D0000672B69930F911F91AF91BF916F917F9105
:106D10000895BF93AF934F939927A42F0E942A2FD2
:106D20000E94A52F4F91AF91BF910895AF93BF934C
:106D3000EF93FF935F936F930F931F932F9310E045
:106D400020E0F5EFEE27509147015F7760914A010F
:106D50006F770491059FA12DE0950491E095069F22
:106D6000B12DA11729F4B21719F4E39591F724C0B6
:106D70001A2F2B2FA0914601B0914901A10FB20FFC
:106D80000E940E31A0914601B0914901A10FB21BA2
:106D90000E940E31A0914601B0914901A11BB21B86
:106DA0000E940E31A0914601B0914901A11BB20F82
:106DB0000E940E31E39569F62F911F910F916F910B
:106DC0005F91FF91EF91DF91AF910895AF93BF93E2
:106DD000EF93FF935F936F930F931F932F933F93C3
:106DE0002FEFF5EFEE27509147015F7760914A0151
:106DF0006F770491059FA12DE0950491E095069F82
:106E0000B12DB21721F4E395A1F73F91D5CF1A2FF9
:106E10002B2FA0914601B09149013A2FB21BA11B23
:106E2000310F0E940E31B20FB20F0E940E31B21B11
:106E3000B21BA3953A17A8F7E395D9F63F91BCCFBB
:106E4000FF91EF91EE0FFF1F5BD03197F695E7951D
:106E50003196EF93FF93C8E7D1E040912C014F9317
:106E6000FF93EF9361D00E94E2300B09205052450E
:106E7000535320454E5445522000EF91FF914F91BE
:106E800040932C0100DC4A3EE9F704DC0E943419EF
:106E90000895FF91EF91EE0FFF1F32D03197F695D5
:106EA000E7953196EF93FF93C8E7D1E040912C012D
:106EB0004F93FF93EF9338D00E94E2300B082028C5
:106EC00059296573202F20284E296F200000EF914B
:106ED000FF914F9140932C01D6DB493761F0493542
:106EE00051F04E3619F04E3409F0F6CFD3DB0E9444
:106EF000341944270895CEDB0E94341941E00895E7
:106F0000C8E7D1E0459146954F93477049934F911B
:106F100042954770499358E145914993403011F0AB
:106F20005A95D1F729920895FF93EF9392E020921A
:106F30002A01A991B991B295B077A770AB0FAA0FAA
:106F4000A0932C01DF93CF930E941519C2E0D8E0E3
:106F5000EBE1FCE00E944732A3E0B9E00E94FB3085
:106F6000CF91DF9158E14991403051F0DF93CF93B9
:106F70005F930E94A62F5F91CF91DF915A9599F769
:106F800040912C01429540932C01EF91FF9108957F
:106F9000FF93EF93DF93CF93BF93AF93C0914601DD
:106FA000D09149010A8119810E3118F4173108F482
:106FB0001AD0A0914801B0914B01C0914601D091E7
:106FC0004901B983AA83AE3138F4B73128F43DD0F2
:106FD0007370713009F076D0AF91BF91CF91DF918E
:106FE000EF91FF910895C0914601D09149010A8126
:106FF00019812C813B81239F310F2596C00DD11D16
:10700000C00DD11D412FE8ECF1E05EE1549FE00D91
:10701000F11DE00FF21D522F699161935A95E1F72E
:107020004395431781F7412FEAE7F4E05EE1549F6F
:10703000E00DF11DE00FF21D522F699161935A95F9
:10704000E1F74395431781F70895C0914601D09128
:1070500049010A8119812C813B81239F310F25969B
:10706000C00DD11DC00DD11D7727412FE8ECF1E0F7
:107070005EE1549FE00DF11DE00FF21D522F619172
:1070800069936F7009F071E05A95C9F743954317FA
:1070900069F7E0914601F09149014081742B7083BA
:1070A000412FEAE7F4E05EE1549FE00DF11DE00FAF
:1070B000F21D522F619169935A95E1F74395431759
:1070C00081F70895C0914601D09149010A81198143
:1070D0002C813B81310F2596412FE8ECF1E05EE1F8
:1070E000549FE00DF11DE00FF21D522F6991619345
:1070F0005A95E1F74395431781F7412FEAE7F4E00A
:107100005EE1549FE00DF11DE00FF21D522F6991D9
:10711000660F28F46E70462E6081607F642961934B
:107120005A95A9F74395431749F70895AF93BF932D
:10713000CF93DF934F935F936F937F934F927091B1
:107140002C014370E1F4A6E0B2E0C4E2D2E0422CAC
:1071500007D0A8EBB4E0C6EDD4E0472E01D061C063
:1071600062E15AE149914D935A95E1F714962496BC
:107170006A95B9F75AE14D925A95E9F70895413069
:10718000C9F4ACE3B4E0CBE3D4E0422C07D0AEEEDC
:10719000B6E0CDEED6E0472E01D043C063E159E121
:1071A0004A914E935A95E1F74E92149725976A9516
:1071B000B1F708954230E1F4ACE3B4E0CEE1D4E0BD
:1071C000422C07D0AEEEB6E0C0EDD6E0472E01D09F
:1071D00028C062E15AE14A914E935A95E1F714971B
:1071E00024976A95B9F75AE14E925A95E9F70895AE
:1071F000A6E0B2E0C7E0D2E0422C07D0A8EBB4E0B2
:10720000C9EBD4E0472E01D00CC063E159E14991AC
:107210004D935A95E1F74D92259614966A95B1F7DC
:1072200008954F907F916F915F914F91DF91CF9132
:10723000BF91AF9108955E984CE54093B80044E843
:107240004093BC0044E94093BC00089544EA0EC05A
:107250005093BB0044E80AC044EC08D05091BB00F6
:10726000089544E803D05091BB0008954093BC00BA
:107270004091BC0047FFFCCF6091B900687F089542
:10728000E5DF683089F4572F550F5E70506AE0DFF4
:10729000683151F45B2FDCDF683231F45A2FD8DFCC
:1072A000683211F4882708958FE0CCCFCFDF6031AA
:1072B000D9F7572F550F5E70516ACADF6034A1F7B6
:1072C00088270895DDDF803049F4F0DF803031F425
:1072D000C8DF683519F411968827B4CF8FE0B2CF94
:1072E0005F93CEDF5F91803031F4B2DF683219F402
:1072F00011968827A7CF8FE0A5CFA8DF6830A9F423
:10730000572F5770550F5169A3DF603471F4A4DF14
:10731000603559F4A52FA5DF683539F4BB27550F23
:10732000AA1F08F4B09588278DCF8FE08BCF8827D0
:10733000D83020F080E34F914F914FEF0895F7DF61
:10734000F999FECFD2BDC1BDF89A40B521960895F6
:10735000EEDFF999FECFD2BDC1BDF89A40B4441614
:1073600011F42196089554E040BDF894FA9AF99AE0
:107370007894F999FECFF89A40B4441511F4219607
:107380000895839580635A9579F70895AF93D7DF71
:107390004193AA95E1F7AF910895AF934191D8DF5A
:1073A000AA95E1F7AF9108954EBD4DB547FFFDCFCA
:1073B0004EB5089588272C9847EDF6DF4427F4DF73
:1073C0002C9A4C7B4432B1F34C31A1F38827443AD8
:1073D00019F04C3909F081E108958827EBDF8030FE
:1073E00021F040E040939C1008954C3911F448E09E
:1073F000F9CF40E1F7CFF1DF403009F40895440FB1
:10740000440F440F440F4A950895AA0FBB1F4B2FFA
:10741000CBDF4A2FC9DF422DC7DFB695A795089568
:10742000803059F44F93C6DF803031F42C9845E515
:10743000BBDFEBDF2C9ABEDF4F910895803059F40B
:107440004F93B8DF803031F42C9843E5ADDFDDDFBA
:107450002C9AB0DF4F910895803051F44F93AADFFA
:10746000803029F42C9846E89FDFCFDF2C9A4F918B
:1074700008951196B0939D10A0939E101197ECCF94
:107480007F93772710D07F9108957F9371E00BD081
:10749000D42F72E008D0C42F7F9108957F9373E0BA
:1074A00002D07F9108958030B9F484DF8030A1F458
:1074B0002C9842ED79DFAA0FBB1FA3954B2F74DFE9
:1074C0004A2F72DF472F70DFB695A7956DDF6CDF0F
:1074D0006BDF6ADF69DF2C9A08958030D1F46ADFB0
:1074E0008030B9F42C9842ED5FDFAA0FBB1F4B2F01
:1074F0005BDF4A2F59DF472F440F56DFB695A7951C
:1075000053DF52DF51DF50DF4FDFD42F4DDFC42F69
:107510002C9A08957F9370E010D07F9108957F9307
:1075200071E04D2F0AD072E04C2FBDDF7F9108959E
:107530007F9373E0B8DF7F9108958030A1F44F937B
:1075400039DF4F91803079F42C984F9347E82CDF46
:1075500044272ADF41E028DF472F26DF4F914F9352
:1075600023DF2C9A4F910895803091F423DF8030EF
:10757000D1F72C984F9347E817DF442715DF40E0F9
:1075800013DF472F11DF4F914F930EDF2C9A4F914E
:1075900008958030D1F4DF93CF934F935F930ADF48
:1075A000803079F42C9847E8FFDE4427FDDE44273D
:1075B000FBDE40E0F9DE55274991F6DE5A95E1F70A
:1075C0002C9A5F914F91CF91DF9108958030B1F463
:1075D0004F935F93EFDE803079F42C9847E8E4DE38
:1075E0004427E2DE4427E0DE40E0DEDE55274FEFB1
:1075F000DBDE5A95E1F72C9A5F914F910895803028
:10760000E1F4DF93CF934F935F93D4DE803089F41E
:107610002C9846EDC9DE4427C7DE4427C5DE40E08E
:10762000C3DE4427C1DE5527BFDE49935A95E1F7F3
:107630002C9A5F914F91CF91DF910895BF93AF93B3
:10764000DF93CF934F935F937F93C7DE403041F436
:107650007F915F914F91CF91DF91AF91BF9108954D
:10766000B5DF4FE057DF442763DFAA27BB27F4DEEF
:1076700011964DEFCA2FCF70C13009F44CEF4ADF9D
:10768000442756DFCC27DD274ADFE6DE1196A030FF
:1076900019F445EE0E94A62F40919C10B41749F7AB
:1076A000D7CFBF93AF93DF93CF934F935F937F93E6
:1076B00094DE403091F47F915F914F91CF91DF91B3
:1076C000AF91BF910895B42FAA271197E7DEC42F79
:1076D000BB27AA27E3DE4C1731F4A2DEDFDE439599
:1076E00027DFBADEE8CF1196D9DE4C17E1F7F5CFE8
:1076F000DF93CF934F9394DE4DEFCA2FCF70C130FD
:1077000009F44CEF07DFC1DE219609DF5FDFA4DE5D
:107710004F91CF91DF910895FF93DF93CF93BF9364
:10772000AF93AA27BB27ED0158DE4030A1F0F42F1C
:10773000A7DE4C3F41F04D3F31F04B3A21F04F3046
:1077400018F0403908F421961196BF1789F744279D
:10775000DF1709F441E0AF91BF91CF91DF91FF9125
:1077600008950F93BF93AF934F93AA27BB27ED01C3
:10777000FD0133DE403099F0042F82DE4D3F49F4A5
:10778000DF93CF9382DE4D2FCF91DF914F3F21F0DA
:1077900021964C3F09F431961196B01771F74F912D
:1077A000AF91BF910F910895FF93EF93DF93CF9324
:1077B0004F932F9312DE4030A9F0AA27BB2760DE3B
:1077C000242FB0919D10A0919E1040910801B417F4
:1077D00010F0A2E0BB27FD0153DE4D3F51F455DE12
:1077E000D21738F42F914F91CF91DF91EF91FF9104
:1077F0000895119640919C10B41709F4BB27BF1748
:1078000059F7AE1749F7AA27BB270ADE39DE4F3FE3
:1078100031F0405F242F7EDE1FDEDF01DDCFAFEFD2
:10782000BFEFE0CFFF93EF93DF93CF93BF93AF937F
:107830004F935F936F937F93D0DD403061F481E18C
:107840007F916F915F914F91AF91BF91CF91DF91F8
:10785000EF91FF91089551D0B41710F08BE1F0CF64
:107860000FDE4C3F11F087E1EBCF40915A014030E1
:1078700011F48BE1E5CF413810F08BE1E1CF71DFFE
:10788000D03021F4C41710F488E1DACFC0E8DBE08F
:1078900050E06FEF69935A95E9F798DE1196B0932F
:1078A0009D10A0939E1040915A01C0E8DBE04F93D9
:1078B0007BDFB993A9934BEA2DDEDF93CF93E5DD10
:1078C00021962DDECF91DF91E9DD32DED2DDE9DEDA
:1078D0004F914A9561F711D0C0E8DBE05ADE409144
:1078E0005C0118DEDF93CF93D0DD219618DECF91B7
:1078F000DF91D4DD1DDEB0DDA3CFA0915801A295AC
:10790000BA2FA07FBF7011960895BF93AF93DF93F6
:10791000CF934F935F937F937727EFDFB1DD4C3F9A
:1079200069F0DBDDDF3F49F0BF93AF93DE01E0DEBE
:10793000AF91BF91B6DE7F5FA1F7DADE7F915F91F5
:107940004F91CF91DF91AF91BF910895BF93AF93C6
:10795000DF93CF934F935F937F932F93AA27BB27F8
:1079600029DD8EDD242FC9DF8BDD4C3F51F489E109
:107970002F917F915F914F91CF91DF91AF91BF9107
:10798000089570915A01703810F08BE1F1CFA5DDA8
:10799000DF3F11F48BE1ECCFDE01CCE3DDE0409181
:1079A0005C01413009F4D395423009F4DE5FF1DD2A
:1079B000DF93CF936ADDD21759F02196B0DDCF91D6
:1079C000DF915EDDA7DD6ADDB3DD46DD6ADED0CFA7
:1079D0008FDEEADE5ADD2196A2DDCF91DF914BEA00
:1079E00099DD5CDDA5DD38DDED0187DF19DD709106
:1079F0005A01770F4D2FB8DD73954C2FB5DD40DD63
:107A000089DD4CDD95DD28DDB3CFBF93AF93DF93E8
:107A1000CF934F935F937F9370DF32DD4C3F49F4F8
:107A20008EE17F915F914F91CF91DF91AF91BF91A7
:107A3000089570915A01703810F08BE1F2CF4DDD4E
:107A4000DF3F11F48BE1EDCFDE01EADCCCE3DDE0DA
:107A500040915C01413009F4D395423009F4DE5F76
:107A6000CEDDDFCF0004080D11161A1F23282C309D
:107A700035393D42464A4F53575B5F64686C7074BA
:107A8000787C7F83878B8F92969A9DA1A4A7ABAEBB
:107A9000B1B5B8BBBEC1C4C6C9CCCFD1D4D6D9DB71
:107AA000DDDFE2E4E6E8E9EBEDEEF0F2F3F4F6F721
:0E7AB000F8F9FAFBFCFCFDFEFEFFFFFFFFFFF6
:107E000000F900F5F3F1F2FC00FAF8F6F4EB5E008D
:107E1000F7000000007131000000797361773200D3
:107E20000063786465343300002076667472350030
:107E3000006E6268677A360000006D6A7537380038
:107E4000002C6B696F303900002E2D6C00707E00A5
:107E500000000000002700000000EA2B00230000C3
:107E6000003C00000000EC0000310034370000004E
:107E7000302C32353638ED00FB2B332D2A390000FB
:107E800000F900F5F3F1F2FC00FAF8F6F4EB00006B
:107E9000F700000000512100000059534157220013
:107EA00000435844452440000020564654522500C3
:107EB000004E4248475A260000004D4A552F2800E0
:107EC000003B4B494F3D2900003A5F4C00503F00BA
:107ED00000000000006000000000EA2A0027000007
:107EE000003E00000000EC000031003437000000CC
:107EF00030E932353638ED00FB2B332D2A390000BE
:107F00000000000000000000000000000000000071
:107F10000000000000000000000000000000000061
:107F20000000000000000000000000000000000051
:107F300000000000000000C000000000000000C1C0
:107F4000000000000000000000002F000000000002
:107F500000000000000000000000EA000000C20075
:107F6000000000000000000000E100E2E00000006E
:107F7000E8E9E500E3E4ED00FB2BE72D2AE600004D
:107F800000000000000000000000000000000000F1
:107F900000000000004000000000000000000000A1
:107FA00000000000000000000000000000000000D1
:107FB000000000000000000000000000007B5B00EB
:107FC00000000000007D5D000000000000007E0059
:107FD00000000000000000000000005C0000000045
:107FE000007C00000000000000E100E2E000000072
:107FF000EFEEE500E3E4ED00FB2BE72D2AE60000C1
:1080000000F900F5F3F1F2FC00FAF8F6F4EB5E008B
:10801000F70000000071310000007A7361773200D0
:10802000006378646534330000207666747235002E
:10803000006E62686779360000006D6A7537380037
:10804000002C6B696F303900002E2F6C3B702D00B7
:10805000000027005B3D00000000EA5D007E00009C
:10806000000000000000EC00003100343700000088
:10807000302C32353638ED00FB2B332D2A390000F9
:1080800000F900F5F3F1F2FC00FAF8F6F4EB000069
:10809000F70000000051210000005A5341574000F2
:1080A00000435844452423000020564654522500DE
:1080B000004E424847595E0000004D4A55262A00AE
:1080C000003C4B494F292800003E3F4C3A505F008E
:1080D000000022007B2B00000000EA7D007C0000F5
:1080E000000000000000EC00003100343700000008
:1080F00030E932353638ED00FB2B332D2A390000BC
:10810000000000000000000000000000000000006F
:10811000000000000000000000000000000000005F
:10812000000000000000000000000000000000004F
:1081300000000000000000C000000000000000C1BE
:10814000000000000000000000002F000000000000
:1081500000000000000000000000EA000000C20073
:10816000000000000000000000E100E2E00000006C
:10817000E8E9E500E3E4ED00FB2BE72D2AE600004B
:1081800000000000000000000000000000000000EF
:1081900000000000000000000000000000000000DF
:1081A00000000000000000000000000000000000CF
:1081B00000000000000000000000000000000000BF
:1081C00000000000000000000000000000000000AF
:1081D000000000000000000000000000000000009F
:1081E000000000000000000000E100E2E0000000EC
:1081F000E8E9E500E3E4ED00FB2BE72D2AE60000CB
:10820000010101010101210101010101013181018E
:108210000100003100010101010131C10101010131
:108220003101010101010131C101010101310101EE
:108230000101010131C1010101011101010101012E
:108240000111C1010101010101010101010101C18E
:10825000010101010101010101000101C10101014F
:10826000010101010101010001C101010101010040
:1082700001010101010141000101010101010100B0
:1082800000000040000000000000000000000000AE
:1082900000000000000000000000000000000000DE
:1082A00000000000000000000000000000000000CE
:1082B00000000000000000000000000000000000BE
:1082C00000000000000000000000000000000000AE
:1082D000000000000000000000000000000000009E
:1082E000100000000000000000000000000000007E
:1082F000200000000000000000000000000000005E
:108300000C11161A1E2225282B2D2F31323333340F
:1083100034343434343434343535363738393B3CFE
:108320003E40434547494B4D4F515253545454548A
:10833000545351504E4C4A4745423F3D3A383634EB
:108340003231302F2E2E2E2F303132333536383A0F
:108350003C3E4042444647494A4B4D4E4E4F50509A
:108360005050505050504F4E4D4C4B494846434151
:108370003E3B37332F2B27221D18130D0802FDF823
:10838000F3EEE9E5E1DDDAD7D4D2D0CECDCCCCCB5B
:10839000CBCBCBCBCBCBCBCBCACAC9C8C7C6C4C34C
:1083A000C1BFBCBAB8B6B4B2B0AEADACABABABABA0
:1083B000ABACAEAFB1B3B5B8BABDC0C2C5C7C9CB1F
:1083C000CDCECFD0D1D1D1D0CFCECDCCCAC9C7C5DB
:1083D000C3C1BFBDBBB9B8B6B5B4B2B1B1B0AFAF30
:1083E000AFAFAFAFAFAFB0B1B2B3B4B6B7B9BCBE59
:1083F000C1C4C8CCD0D4D8DDE2E7ECF2F7FD020767
:10840000000A141D272F383F464B505457595959CD
:10841000585654504C48433E39332E2925201C19B8
:1084200016141211111112131517191C1F222527CA
:108430002A2C2E303132323232312F2D2B28252268
:108440001F1C191613110F0D0C0B0A0A0A0B0C0E28
:1084500010121416181A1C1E1F2020201F1E1C1973
:1084600016120D0803FDF7F0EAE3DDD6D1CBC6C244
:10847000BFBDBBBABBBCBEC2C6CBD1D7DFE6EFF730
:108480000008101920282E34393D41434445444208
:10849000403D39342E29221C150F0802FCF7F2ED5D
:1084A000E9E6E3E1E0DFDFDFE0E1E3E5E7E9EBED8B
:1084B000EFF1F3F4F5F5F5F4F3F2F0EEECE9E6E3C1
:1084C000E0DDDAD7D4D2D0CECDCDCDCDCECFD1D385
:1084D000D5D8DADDE0E3E6E8EAECEDEEEEEEEDEB42
:1084E000E9E6E3DFDAD6D1CCC6C1BCB7B3AFABA9FE
:1084F000A7A6A6A6A8ABAFB4B9C0C7D0D8E2EBF583
:1085000080675342352B221C16120E0C09070605F4
:108510000400000000000000000000000000000057
:10852000000000000000000000000000000000004B
:10853000000000000000000000000000000000003B
:10854000000000000000000000000000000000002B
:10855000000000000000000000000000000000001B
:10856000000000000000000000000000000000000B
:1085700000000000000000000000000000000000FB
:10858000890091009A00A300AD00B700C200CE00A0
:10859000DA00E700F400030112012301340146016F
:1085A0005A016E0184019B01B301CD01E90106026C
:1085B0002502450268028C02B302DC02080336037E
:1085C00067039B03D2030C0449048B04D0041905F0
:1085D0006705B90510066C06CE063507A307170810
:1085E000930815099F09320ACD0A720B200CD80C8A
:1085F0009C0D6B0E460F2F1025112A123F13641489
:10860000008A0A80008A0A80008A0A80008A0A801A
:10861000EC24248002C0084A242424000000000026
:10862000000000000000000000000000000000004A
:10863000000000000000000000000000000000003A
:10864000000000000000000000000000000000002A
:10865000000000000000000000000000000000001A
:10866000000000000000000000000000000000000A
:1086700000000000000000000000000000000000FA
:1086800024C002C00004620000000000000000805E
:10869000C0A2868200000000000000002286ECAA32
:1086A0000024000006A28080000002C02480002078
:1086B00000008000000042248000C002C20C0000C4
:1086C000000080000000000000000000000000002A
:1086D000808A808006A282408080C6A000004482FA
:1086E0000000000000008000C002EC0E0080242486
:1086F0002400000024240024242424000026E48AEA
:10870000008A0A80008A0A80008A0A80008A0A8019
:108710006C424280A4A4084A464242002000000065
:10872000000C2C2C0C4A242404280000000000001B
:10873000200C204004400840202000000400282095
:10874000202042204240402060200A606260602079
:1087500042204220406060606060404600460C005D
:108760002800620002000800620C0462240000007D
:108770000000000028000000000000040C28620037
:1087800024A202C0660A8A000000000000000080E7
:10879000C0A28682000000000000008040826C4C75
:1087A0000C2400000A8A808002C002C024EC246CE1
:1087B00000420400000042E68000C002C220000027
:1087C000246CC20000000000000000000000000057
:1087D0008086A00A0A8A8240C002C6A00000848067
:1087E000000000808000C08AE044EC440000204685
:1087F0002400000024240024242424000026E4C0B3
:10880000008A0A80008A0A80008A0A80008A0A8018
:10881000EC4242808080084A424242242C00000000
:10882000000C2C2C2248660C0C0C0C0C00000002D6
:108830006024600408622860606024240C000C60DE
:108840006060606060626260600C0466624C6060E0
:10885000606060600C60606060600262000C2C0010
:108860000C00620002002A00620000620C0000009E
:1088700000000000280000000000000C0C0C620C3E
:10888000428A06A2800A8A000000000000000080E0
:10889000C0A2868200000000000080804082ECAA16
:1088A0002024242422868080A0A2046242804240A8
:1088B00000420440824242800000C0026620004222
:1088C000266CC28080000000000000000000000054
:1088D0008082ACA822868622CC2AC6A040828480D0
:1088E000000000C2C242C00CEC0EEC0E00802286DA
:1088F0002400000024240024242424000026E4A2D0
:10890000008A0A80008A0A80008A0A80008A0A8017
:108910006C80808080800A8A82808042200C602067
:10892000000C2C406E046E2828046C0C000000041F
:10893000640C020C2C42620460602424284004026F
:108940000260606260626262600C046E626C486029
:10895000606060620C6060602C600462280C6000E3
:1089600004204220262028226A2408660C4E6A2011
:1089700046206A20466060606060400C0C0C280451
:1089800042860A8A80046200000000000000008025
:10899000C0A28682000000000080808080806CE69B
:1089A00040424242228640828AA2046242EC246013
:1089B00000420440824242240000C002662000803F
:1089C000E620C280C200000000000000000000009D
:1089D0008080AC0A40828622E426C6A08080448241
:1089E000000000C2E642E004EC44E044008022863D
:1089F0002400000024240024242424000026E4E091
:108A0000008A0A80008A0A80008A0A80008A0A8016
:108A1000EC808080A88C0A8A80E6E642002C6060A8
:108A2000000C002C200C2800280420400040000CE2
:108A30006C0C04046602420C202200006200020456
:108A40002660426260424268400C044A626C6C607C
:108A5000426042200C6060600C2C0C626C0C0000C8
:108A60000002606264604660480C046E0C6C4860F2
:108A700066664862286060602C6004280C040C80E4
:108A800080820A8A66046200000000000000008004
:108A9000C0A2868200000000808080808080ECAAD6
:108AA0000C8042244082408280820C2880802420D6
:108AB00000420440824242420000C00224200C8056
:108AC000E020CA80C200000000000000000000009A
:108AD000A0A8AC4080808080E426C6A0860A4082A0
:108AE000000000C2E642EC2AEC60C00280802286D0
:108AF0002480228622868080228680228626E4E8C0
:108B0000000000008A8A8A8A0A0A0A0A8080808015
:108B10006C8080800A8AA88C40808042004060601F
:108B2000000C00400E286E0028046C0C2400002865
:108B3000480C0C024002600C600224242840040C03
:108B40006C40606260626260600C046E62606460CF
:108B5000626C6E020C602C6C2C0C2862040C000001
:108B60000022606260402860600C044A0C6C606007
:108B700066666220286060600C260C0C0C0C0404F5
:108B800080822286660462000000000000000080EF
:108B9000C0A28682000000008080808080806CE619
:108BA0000C008042408240828080280C80EC800C47
:108BB00000428040824242420000C0022400204223
:108BC0004620C280C200000000000000000000003B
:108BD000ACCAA00A82404082E426C6A044828080BB
:108BE000000000C2E642EC2AE044C00280802286F7
:108BF0002480228622868080228680228626E42483
:108C0000000000008A8A8A8A0A0A0A0A8080808014
:108C1000EC8080800A8A808082C2A4420000602C9E
:108C20000000002C426466000C0C0C0C0C0024624A
:108C3000600C2860046060286004240C0C000C00A8
:108C40006C60606060626260600C6666626060605A
:108C5000626466600C602C6C600C6262000C000048
:108C60000060606060622822600C046E0C606060CE
:108C7000462062022C642C6C2C06280C0C0C020C76
:108C800042862286800A8A000000000000000080E0
:108C9000C0A2868200000080808080808080ECAA54
:108CA00040008080408222868082280CCE80244032
:108CB00000426240824242240000C002660020C29C
:108CC0002420C280C200000000000000000000005C
:108CD000ACA8808082402286E044C2C24482808068
:108CE000000000C2E642EC2AC002C0028000242438
:108CF0002400242400002400242424228626E4289E
:108D0000000000008A8A8A8A0A0A0A0A8080808013
:108D10006C428042084A808042E642240000424C75
:108D2000000C002C0C06260004280000280024005B
:108D30002020402004202028202400280400280C83
:108D40002060422042406220602024604060602019
:108D5000622660200C200C20600C4046004600403B
:108D600000224220202028026020666620606020C9
:108D7000620462420C260C2C600240040C280200A3
:108D8000428A4082800A8A000000000000000080C1
:108D9000C0A28682000080808080808040826C4CEF
:108DA00020008024808022868AA26204CEEC420CBD
:108DB00000426240824242E60000C002660020009B
:108DC0002440C2808000000000000000000000007D
:108DD000ACA8808080800A8ACA88C00284804082D1
:108DE000000000C2C242E02AC00280808000242429
:108DF0002400242400002400242424228626E4289D
:108E0000000000008A8A8A8A0A0A0A0A8080808012
:108E1000EC428042084AA4A4408042000000620064
:108E20000000000000000000000000000000000042
:108E30000000000000000000000000000000000032
:108E40000000000000000000000000000000000022
:108E50000000000000000000000000000000000012
:108E600000000000000000200000240000000000BE
:108E7000620600000000000000200000000000006A
:108E800024A28080660462000000000000000080D0
:108E9000C0A2868200808080808080804082ECE654
:108EA0000C00424280800A8AA0A2C002CE80662CBA
:108EB00000426200004200800080C002C200200028
:108EC0004240C2000000000000000000000000005E
:108ED000A0A88080824006A2C6A080808480000076
:108EE000000000808000C02AC0020000000024248E
:108EF0002400242400002400242424204626E40006
:108F0000000000008A8A8A8A0A0A0A0A8080808011
:108F10006C248024084A0A8A80E624000000C000ED
:108F20000000000000000000000000000000000041
:108F30000000000000000000000000000000000031
:108F40000000000000000000000000000000000021
:108F50000000000000000000000000000000000011
:108F60000000000000000000000000000000000001
:108F700000000000000000000000000000000000F1
:108F800024C0808000046200000000000000008017
:108F9000C0A28682808080808080808022866C4C07
:108FA00000004280808006A202C0C00284ECA44C73
:108FB00000006200004200240080C002C2000000E5
:108FC0000000800000000000000000000000000021
:108FD0008080000082400000C6A000004620000003
:108FE000000000000000C002E044000080002424D3
:108FF0002400242400002400242424242426E40023
:0C900000202020202020202020202020E4
:0C9C0000202020202020202020202020D8
:0CA80000202020202020202020202020CC
:0CB40000202020202020202020202020C0
:0CC00000202020202020202020202020B4
:0CCC0000202020202020202020202020A8
:0CD800002020202020202020202020209C
:0CE4000020202020202020202020202090
:10F0000040913C01C8EFD7E00E94A83940910C0123
:10F010000E94A83940910D010E94A8390895C8EFB7
:10F02000D7E00E949F39427040933C010E949F3973
:10F03000417040930C010E949F39417040930D0133
:10F040000895FF93EF93DF93CF93AF93F2D0E093C4
:10F050003401F0933501AF91CF91DF91EF91FF91A2
:10F060000895E0E0F0E9C0E0DCE0A42FA03021F05A
:10F07000EC0FFD1FAA95FACF0895E0913401F091AD
:10F080003501A0E2A99FE00DF11DB096C0EAD1E0E4
:10F09000A0E2B591B993AA95E1F7BFEFB9930895AE
:10F0A00047B740FDFDCFB7BFE89547B740FDFDCF5F
:10F0B000089547B746FF0895B1E1F2DFFACFF8941B
:10F0C0004E2F407E19F4B3E0EBDFF3DFA0E10990AF
:10F0D0001990B1E0E5DF3296AA95C9F7E03009F062
:10F0E00008953297B5E0DCDFE4DF32960895F894B6
:10F0F0004F93BF93AF93B3E0D3DFDBDF3297CCE323
:10F10000DFE0A0E8329609901990B1E0C9DFAA9536
:10F11000C9F7B5E0C5DFCDDFAF91BF914F9108953D
:10F12000E0913401F0913501B097ACE0B591B9931D
:10F13000AA95E1F7A0912901A7FD0895A6EAB2E0FA
:10F14000CA0FDB1FACE0B0912C01B993AA95E9F787
:10F150000895E0E0F0E9A0E0BCE0492F403029F359
:10F16000EA0FFB1F4A95FACFF89461D0C0EAD1E0CC
:10F17000A3EDB1E05CE04D9149935A95E1F754E17C
:10F1800040E2B9935A95E9F7A09799DF9927B3E23E
:10F19000B99FA4E3B2E0A00DB11DC8E7D1E050E2F1
:10F1A0004D9149935A95E1F7299250E24A914032A4
:10F1B00019F428825A95D1F70E947D17C0EAD1E050
:10F1C0007EDF93959F3519F77894089530D0A3ED9D
:10F1D000B1E05CE045914D935A95E1F7749699271B
:10F1E00050E2A0EAB1E045914D935A95E1F7A8E7C6
:10F1F000B1E040E253E24D935A95E9F7FF93EF9364
:10F200009F930E9467189F91EF91FF91C8E7D1E00B
:10F21000B3E2B99FA1E3B2E0A00DB11D53E2499161
:10F220004D935A95E1F793959F35D1F60895409106
:10F230003D01E0E0F0E947704295A0ECA49FE00DAD
:10F24000F11D0895CCE3DFE040E250E259934A9586
:10F25000E9F740EF5FEF59934A95E9F7E8DF47DFB9
:10F260003296CCE3DFE040E25FEF59934A95E9F74D
:10F270004BE04F933CDF32964F914A95D1F778940B
:10F280000895472F4770D5DFFF93EF93D0DFAF91FD
:10F29000BF914CE04F93CCE3DFE040E055915993B0
:10F2A0004A95E1F7FF93EF93FD0121DF3296DF01ED
:0EF2B000EF91FF914F914A9569F77894089578
:10F50000FFFFFFFFFFFFFFFFFFFFFFFEFEFEFEFE10
:10F51000FEFEFDFDFDFDFDFCFCFCFCFBFBFBFBFA28
:10F52000FAFAF9F9F9F8F8F8F7F7F6F6F6F5F5F466
:10F53000F4F3F3F2F2F2F1F0F0EFEFEEEEEDEDECCA
:10F54000EBEBEAEAE9E8E8E7E6E6E5E4E4E3E2E152
:10F55000E1E0DFDEDEDDDCDBDADAD9D8D7D6D5D400
:10F56000D4D3D2D1D0CFCECDCCCBCAC9C9C8C7C6CF
:10F57000C5C4C3C2C1BFBEBDBCBBBAB9B8B7B6B5BE
:10F58000B4B2B1B0AFAEADACAAA9A8A7A6A5A3A2CC
:10F59000A1A09E9D9C9B99989796949392918F8EF3
:10F5A0008D8B8A898786858382817F7E7D7B7A7831
:10F5B0007776747371706F6D6C6A69676665636284
:10F5C000605F5D5C5A595756545351504E4D4B4AEB
:10F5D0004847454442413F3E3C3B3938363533325B
:10F5E000302E2D2B2A2827252422201F1D1C1A19D6
:10F5F00017161412110F0E0C0B0907060403010055
:10F6000000A0208000A0208000A0208000A02080FA
:10F610006C484880040024A04848480000000000CE
:10F6200000000000000000000000000000000000DA
:10F6300000000000000000000000000000000000CA
:10F6400000000000000000000000000000000000BA
:10F6500000000000000000000000000000000000AA
:10F66000000000000000000000000000000000009A
:10F67000000000000000000000000000000000008A
:10F680008020A0008020A0008020A0008020A0007A
:10F69000ECC8C8008480A420C8C8C880808080804E
:10F6A000808080808080808080808080808080805A
:10F6B000808080808080808080808080808080804A
:10F6C000808080808080808080808080808080803A
:10F6D000808080808080808080808080808080802A
:10F6E000808080808080808080808080808080801A
:10F6F000808080808080808080808080808080800A
:10F7000000A0208000A0208000A0208000A02080F9
:10F71000EC848480C8C824A088848400440000004D
:10F7200000286C6C28A048480C6000000000000015
:10F73000442844800C802480444400000C00604431
:10F740004444844484808044C44420C4C0C4C44429
:10F750008444844480C4C4C4C4C48088008828000D
:10F760006000C00004002400C0280CC04800000055
:10F7700000000000600000000000000C2860C000D5
:10F780008020A0008020A0008020A0008020A00079
:10F790006C0404004848A42008040480C4808080CD
:10F7A00080A8ECECA820C8C88CE080808080808095
:10F7B000C4A8C4008C00A400C4C480808C80E0C4B1
:10F7C000C4C404C4040000C444C4A044404444C4A9
:10F7D00004C404C400444444444400088008A8808D
:10F7E000E08040808480A48040A88C40C8808080D5
:10F7F00080808080E08080808080808CA8E0408055
:10F8000000A0208000A0208000A0208000A02080F8
:10F810006C848480808024A0848484486C000000F0
:10F8200000286C6C40A4CC2828282828000000045C
:10F83000C448C40C24C060C4C4C44848280028C4B8
:10F84000C4C4C4C4C4C0C0C4C4280CCCC0A8C4C4EC
:10F85000C4C4C4C428C4C4C4C4C404C000286C0044
:10F860002800C00004006400C00000C028000000A0
:10F870000000000060000000000000282828C028C8
:10F880008020A0008020A0008020A0008020A00078
:10F89000EC0404000000A420040404C8EC80808070
:10F8A00080A8ECECC0244CA8A8A8A8A880808084DC
:10F8B00044C8448CA440E0444444C8C8A880A84438
:10F8C000444444444440404444A88C4C402844446C
:10F8D00044444444A84444444444844080A8EC80C4
:10F8E000A88040808480E48040808040A880808020
:10F8F00080808080E0808080808080A8A8A840A848
:10F9000000A0208000A0208000A0208000A02080F7
:10F91000EC808080808020A0848080844428C4443F
:10F9200000286C80E80CE860600CEC280000000CFB
:10F93000C82804286C84C00CC4C4484860800C04E7
:10F9400004C4C4C0C4C0C0C0C4280CE8C0ECA4C473
:10F95000C4C4C4C028C4C4C46CC40CC06028C400DF
:10F960000C4484444C446040E44824CC28ACE44437
:10F970008844E44488C4C4C4C4C480282828600CD3
:10F980008020A0008020A0008020A0008020A00077
:10F990006C0000000000A02004000004C4A844C4BF
:10F9A00080A8EC00688C68E0E08C6CA88080808C7B
:10F9B00048A884A8EC04408C4444C8C8E0008C8467
:10F9C000844444404440404044A88C68406C2444F3
:10F9D00044444440A8444444EC448C40E0A844805F
:10F9E0008CC404C4CCC4E0C064C8A44CA82C64C4B7
:10F9F00008C464C408444444444400A8A8A8E08C53
:10FA000000A0208000A0208000A0208000A02080F6
:10FA10006C808080E0A820A0804C4C84006CC4C422
:10FA20000028006C44286000600C4480008000289E
:10FA3000EC280C0CCC04842844400000C000040CCA
:10FA40004CC484C0C48484E080280CA0C0ECECC406
:10FA500084C4844428C4C4C4286C28C0EC28000092
:10FA60000004C4C0C8C488C4A4280CE828ECA4C4FA
:10FA7000CCCCA4C060C4C4C46CC40C60280C288066
:10FA80008020A0008020A0008020A0008020A00076
:10FA9000EC0000006028A02000CCCC0480EC4444A2
:10FAA00080A880ECC4A8E080E08CC400800080A81E
:10FAB0006CA88C8C4C8404A8C4C080804080848C4A
:10FAC000CC4404404404046000A88C20406C6C4486
:10FAD000044404C4A8444444A8ECA8406CA8808012
:10FAE000808444404844084424A88C68A86C24447A
:10FAF0004C4C2440E0444444EC448CE0A88CA800E6
:10FB000000000000A0A0A0A02020202080808080F5
:10FB1000EC80808020A0E0A8808080840080C4C425
:10FB2000002800802C60E800600CEC284800006091
:10FB3000A42828048004C428C404484860800C28F1
:10FB4000EC80C4C0C4C0C0C4C4280CE8C0C4C8C4CD
:10FB5000C0ECE80428C46CEC6C2860C00C280000E1
:10FB60000040C4C0C48060C4C4280CA028ECC4C435
:10FB7000CCCCC04460C4C4C4284C282828280C0C11
:10FB80008080808020202020A0A0A0A00000000075
:10FB90006C000000A02060280000000480004444A5
:10FBA00080A88000ACE06880E08C6CA8C88080E011
:10FBB00024A8A884008444A84484C8C8E0008CA871
:10FBC0006C0044404440404444A88C68404448444D
:10FBD000406C6884A844EC6CECA8E0408CA8808061
:10FBE00080C044404400E04444A88C20A86C4444B5
:10FBF0004C4C40C4E0444444A8CCA8A8A8A88C8C91
:10FC000000000000A0A0A0A02020202080808080F4
:10FC10006C80808020A080808404C8840000C46C34
:10FC20000000006C84C8CC0028282828280048C080
:10FC3000C42860C40CC4C460C40C48282800280030
:10FC4000ECC4C4C4C4C0C0C4C428CCCCC0C4C4C4E4
:10FC5000C0C8CCC428C46CECC428C0C000280000B4
:10FC600000C4C4C4C4C06040C4280CE828C4C4C4D0
:10FC70008844C0046CC86CEC6C08602828280428F0
:10FC80008080808020202020A0A0A0A00000000074
:10FC9000EC000000A020000004844804808044ECB4
:10FCA000808080EC04484C80A8A8A8A8A880C84000
:10FCB00044A8E0448C4444E0448CC8A8A880A880B0
:10FCC0006C4444444440404444A84C4C4044444464
:10FCD00040484C44A844EC6C44A8404080A8808034
:10FCE000804444444440E0C044A88C68A844444450
:10FCF00008C44084EC48EC6CEC88E0A8A8A884A870
:10FD000000000000A0A0A0A02020202080808080F3
:10FD1000EC84808424A08080844C8448000084A8E3
:10FD20000028006C28084C000C60000060004800AF
:10FD3000444480440C444460444800600C00602803
:10FD400044C484448480C044C44448C480C4C4447B
:10FD5000C04CC44428442844C428808800880080BB
:10FD60000040844444446004C444CCCC44C4C444EF
:10FD7000C00CC084284C286CC404800C286004008B
:10FD80008080808020202020A0A0A0A00000000073
:10FD90006C040004A420000004CC04C88080042863
:10FDA00080A880ECA888CC808CE08080E080C8802F
:10FDB000C4C400C48CC4C4E0C4C880E08C80E0A883
:10FDC000C44404C4040040C444C4C844004444C4FB
:10FDD00040CC44C4A8C4A8C444A80008800880003B
:10FDE00080C004C4C4C4E08444C44C4CC44444C46F
:10FDF000408C4004A8CCA8EC4484008CA8E084800B
:10FE000000000000A0A0A0A02020202080808080F2
:10FE10006C84808424A0C8C8808084000000C00056
:10FE200000000000000000000000000000000000D2
:10FE300000000000000000000000000000000000C2
:10FE400000000000000000000000000000000000B2
:10FE500000000000000000000000000000000000A2
:10FE60000000000000000044000048000000000006
:10FE7000C008000000000000004400000000000076
:10FE80008080808020202020A0A0A0A00000000072
:10FE9000EC040004A42048480000048080804080D6
:10FEA0008080808080808080808080808080808052
:10FEB0008080808080808080808080808080808042
:10FEC0008080808080808080808080808080808032
:10FED0008080808080808080808080808080808022
:10FEE00080808080808080C48080C8808080808086
:10FEF000408880808080808080C4808080808080F6
:10FF000000000000A0A0A0A02020202080808080F1
:10FF1000EC48804824A020A0804C4800000000004D
:10FF200000000000000000000000000000000000D1
:10FF300000000000000000000000000000000000C1
:10FF400000000000000000000000000000000000B1
:10FF500000000000000000000000000000000000A1
:10FF60000000000000000000000000000000000091
:10FF70000000000000000000000000000000000081
:10FF80008080808020202020A0A0A0A00000000071
:10FF90006CC800C8A420A02000CCC88080808080CD
:10FFA0008080808080808080808080808080808051
:10FFB0008080808080808080808080808080808041
:10FFC0008080808080808080808080808080808031
:10FFD0008080808080808080808080808080808021
:10FFE0008080808080808080808080808080808011
:10FFF0008080808080808080808080808080808001
:00000001FF
